:020000040800F2
:1000000000060020B5050008ED3100086D3100083C
:10001000C53100086D31000899310008B7050008A6
:10002000B7050008B7050008B705000841400008FB
:10003000B7050008B7050008B7050008B7050008B0
:10004000B7050008B7050008B7050008B7050008A0
:10005000B7050008B7050008BD6E0008E96E000886
:10006000156F0008416F00086D6F0008B7050008A4
:10007000B7050008B7050008B7050008B705000870
:10008000B7050008B7050008B7050008B52D00083A
:10009000DD2D0008C92D0008F12D0008996F00081A
:1000A000B7050008B7050008B7050008B705000840
:1000B000B7050008B7050008B7050008B705000830
:1000C000B7050008B7050008B7050008B705000820
:1000D000B7050008B7050008B7050008B705000810
:1000E000FD6F0008B7050008B7050008B705000850
:1000F000B7050008B7050008B7050008B7050008F0
:10010000B7050008B705000885700008B7050008A6
:10011000B7050008B7050008B7050008B7050008CF
:10012000B7050008B7050008B7050008B7050008BF
:10013000B7050008B7050008B7050008B7050008AF
:10014000B7050008B7050008B7050008B70500089F
:10015000B7050008B7050008B7050008B70500088F
:10016000B7050008B7050008B7050008B70500087F
:10017000B7050008E5650008B7050008B7050008E1
:10018000B7050008B705000871700008B70500083A
:10019000B7050008B7050008B7050008B70500084F
:1001A000B7050008B7050008B7050008B70500083F
:1001B000B7050008B7050008B7050008B70500082F
:1001C000B7050008B7050008B7050008B70500081F
:1001D000B7050008D1650008B7050008B705000895
:1001E000B7050008B7050008B7050008B7050008FF
:1001F000B7050008B7050008B7050008B7050008EF
:10020000B7050008B7050008B7050008B7050008DE
:10021000B7050008B7050008B7050008B7050008CE
:10022000B7050008B7050008B7050008B7050008BE
:10023000B7050008B7050008B7050008B7050008AE
:10024000B7050008B7050008B7050008B70500089E
:10025000B7050008B7050008B7050008B70500088E
:10026000B7050008B7050008B7050008B70500087E
:10027000B7050008B7050008B7050008B70500086E
:10028000B7050008B7050008B7050008B70500085E
:10029000B7050008B7050008B7050008B70500084E
:1002A000391A0008000000000000000000000000F3
:1002B00053B94AB9002908BF00281CBF4FF0FF31CD
:1002C0004FF0FF3000F074B9ADF1080C6DE904CEC9
:1002D00000F006F8DDF804E0DDE9022304B0704721
:1002E0002DE9F047089D04468E46002B4DD18A42E9
:1002F000944669D9B2FA82F252B101FA02F3C2F11C
:10030000200120FA01F10CFA02FC41EA030E9440AC
:100310004FEA1C48210CBEFBF8F61FFA8CF708FBCD
:1003200016E341EA034306FB07F199420AD91CEBA5
:10033000030306F1FF3080F01F81994240F21C81D7
:10034000023E63445B1AA4B2B3FBF8F008FB10331F
:1003500044EA034400FB07F7A7420AD91CEB040454
:1003600000F1FF3380F00A81A74240F20781644424
:10037000023840EA0640E41B00261DB1D4400023A9
:10038000C5E900433146BDE8F0878B4209D9002D0D
:1003900000F0EF800026C5E9000130463146BDE897
:1003A000F087B3FA83F6002E4AD18B4202D3824201
:1003B00000F2F980841A61EB030301209E46002DB0
:1003C000E0D0C5E9004EDDE702B9FFDEB2FA82F205
:1003D000002A40F09280A1EB0C014FEA1C471FFA63
:1003E0008CFE0126200CB1FBF7F307FB131140EA4A
:1003F00001410EFB03F0884208D91CEB010103F117
:10040000FF3802D2884200F2CB804346091AA4B2D8
:10041000B1FBF7F007FB101144EA01440EFB00FEAC
:10042000A64508D91CEB040400F1FF3102D2A64511
:1004300000F2BB800846A4EB0E0440EA03409CE7B0
:10044000C6F12007B34022FA07FC4CEA030C20FA5D
:1004500007F401FA06F31C43F9404FEA1C4900FA7D
:1004600006F3B1FBF9F8200C1FFA8CFE09FB1811FA
:1004700040EA014108FB0EF0884202FA06F20BD96D
:100480001CEB010108F1FF3A80F08880884240F2BD
:100490008580A8F102086144091AA4B2B1FBF9F001
:1004A00009FB101144EA014100FB0EFE8E4508D9FC
:1004B0001CEB010100F1FF346CD28E456AD9023881
:1004C000614440EA0840A0FB0294A1EB0E01A14266
:1004D000C846A64656D353D05DB1B3EB080261EBD4
:1004E0000E0101FA07F722FA06F3F1401F43C5E9AE
:1004F000007100263146BDE8F087C2F12003D840E4
:100500000CFA02FC21FA03F3914001434FEA1C4725
:100510001FFA8CFEB3FBF7F007FB10360B0C43EA17
:10052000064300FB0EF69E4204FA02F408D91CEBC7
:10053000030300F1FF382FD29E422DD902386344C5
:100540009B1B89B2B3FBF7F607FB163341EA034165
:1005500006FB0EF38B4208D91CEB010106F1FF38B4
:1005600016D28B4214D9023E6144C91A46EA0046AB
:1005700038E72E46284605E70646E3E61846F8E63D
:100580004B45A9D2B9EB020864EB0C0E0138A3E786
:100590004646EAE7204694E74046D1E7D0467BE767
:1005A000023B614432E7304609E76444023842E7DF
:1005B000704700BF02E000F000F8FEE772B63A486C
:1005C00080F30888394880F3098839484EF6085185
:1005D000CEF20001086040F20000CCF200004EF6BE
:1005E0003471CEF200010860BFF34F8FBFF36F8FFD
:1005F00040F20000C0F2F0004EF68851CEF2000149
:100600000860BFF34F8FBFF36F8F4FF00000E1EE34
:10061000100A4EF63C71CEF200010860062080F30D
:100620001488BFF36F8F05F0E5FA05F087FA06F03E
:100630000BFA4FF055301F491B4A91423CBF41F81D
:10064000040BFAE71C49194A91423CBF41F8040BDC
:10065000FAE71A491A4A1B4B9A423EBF51F8040B5B
:1006600042F8040BF8E700201749184A91423CBFB2
:1006700041F8040BFAE705F09FFA06F05DFA144C16
:10068000144DAC4203DA54F8041B8847F9E700F034
:1006900041F8114C114DAC4203DA54F8041B884761
:1006A000F9E705F087BA00000006002000220020CC
:1006B00000000008000000200006002070770008FD
:1006C00000220020C8220020C82200202082002012
:1006D000A0020008A4020008A4020008A402000866
:1006E0002DE9F04F2DED108AC1F80CD0D0F80CD0C8
:1006F000BDEC108ABDE8F08F002383F311882846F3
:10070000A047002004F066FDFEE704F0D5FC00DF02
:10071000FEE70000F8B501F0CFFA30B1264B002219
:100720000E211A725A729972DA7205F08BF9074625
:1007300005F0FAF90546A0BB204B9F4231D00133AA
:100740009F4231D027F0FF021D4B9A422FD12E46F7
:1007500042F21074F8B200F09FFD00F0A7FF08B15C
:100760000024264600F09EFD08B90646044635B131
:10077000144B9F4203D0002405F0CEF926460020FA
:1007800005F06AF90EB100F065F801F019FB00F010
:10079000B1FF01F0D7F9204600F012F900F05AF845
:1007A000F9E72E460024D8E704460126D5E7064699
:1007B00041F28834D1E700BF00220020010007B0D9
:1007C000000008B0263A09B008B501F087F9A0F199
:1007D00020035842584108BD07B541F212030221D7
:1007E00001A8ADF8043001F097F903B05DF804FBFF
:1007F000202310B583F311881248C3680BB104F0AD
:100800006FFD0023104A4FF47A710E4804F02CFD5E
:10081000002383F311880D4C236813B12368013B37
:100820002360636813B16368013B6360084B1B7806
:1008300033B9636823B9022001F044FA32236360BC
:1008400010BD00BFC8220020F1070008E4230020EB
:10085000DC220020F8B5534B534A1C46196801317D
:1008600000F09F8004339342F8D162684F4B9A4264
:1008700040F297804E4B9B6803F1006303F5003311
:100880009A4280F08E8005F01BF905F02DF90020CA
:1008900001F072F90220474B187001F011FA464B33
:1008A0000021D3F8E820C3F8E810D3F81021C3F8EA
:1008B0001011D3F81021D3F8EC20C3F8EC10D3F8C2
:1008C0001421C3F81411D3F81421D3F8F020C3F87D
:1008D000F010D3F81821C3F81811D3F81821D3F861
:1008E000802042F00062C3F88020D3F8802022F0FC
:1008F0000062C3F88020D3F88020D3F8802042F033
:100900000072C3F88020D3F8802022F00072C3F870
:100910008020D3F8803072B64FF0E023C3F8084D42
:10092000D4E90004BFF34F8FBFF36F8F234AC2F89F
:100930008410BFF34F8F536923F480335361BFF3A7
:100940004F8FD2F8803043F6E076C3F3C905C3F386
:100950004E335B0103EA060C29464CEA81770139E4
:10096000C2F87472F9D2203B13F1200FF2D1BFF319
:100970004F8FBFF36F8FBFF34F8FBFF36F8F5369ED
:1009800023F4003353610023C2F85032BFF34F8F7A
:10099000BFF36F8F202383F31188854680F3088887
:1009A0002047F8BD0000020820000208FFFF0108F0
:1009B00000220020DC2200200044025800ED00E06C
:1009C0002DE9F04F93B0AC4B2022FF2100900AA8F4
:1009D0009D6801F09FF9A94A1378A3B90121A8489D
:1009E0001170C360202383F31188C3680BB104F036
:1009F00077FC0023A34A4FF47A71A14804F034FC39
:100A0000002383F31188009B9F4A03B113600023E6
:100A10009E49009C98469B461E469A460B70536022
:100A2000012001F04DF924B1974B1B68002B00F019
:100A30001C82002001F052F80390039B002B01DA86
:100A400000F0A8FE039B002BEDDB012001F036F93E
:100A5000039B213B162BE3D801A252F823F000BFE1
:100A6000BD0A0008E50A0008790B0008210A000801
:100A7000210A0008210A00080D0C0008DF0D0008FB
:100A8000F90C00085B0D0008830D0008A90D000893
:100A9000210A0008BB0D0008210A00082D0E0008DD
:100AA0005D0B0008210A0008710E0008C90A000841
:100AB0005D0B0008210A00085B0D00080220FFF70B
:100AC00083FE002840F0FB81009B022105A8B8F1BD
:100AD000000F08BF1C4641F21233ADF8143001F08C
:100AE0001BF89DE74FF47A7000F0F8FF071EEBDB70
:100AF0000220FFF769FE0028E6D0013F052F00F233
:100B0000E081DFE807F0030A0D1013360523042106
:100B100005A8059301F000F817E004215648F9E70D
:100B200004215B48F6E704215A48F3E74FF01C091B
:100B3000484609F1040901F021F80421059005A8AF
:100B400000F0EAFFB9F12C0FF2D101204FF0000ABA
:100B500000FA07F747EA0B0B5FFA8BFB01F026F967
:100B600026B10BF00B030B2B08BF0024FFF734FE5C
:100B700056E704214848CDE7002EA5D00BF00B0323
:100B80000B2BA1D10220FFF71FFE074600289BD0A8
:100B900001203E4E00F0F0FF4FF0000802203070C0
:100BA00001F08EF85FFA88F9484600F0F5FF044638
:100BB00090B1484608F1010800F0FEFF0028F1D18D
:100BC000B846044641F21213022105A83E46ADF88C
:100BD000143000F0A1FF23E70123254602203370E3
:100BE00001F06CF8244B9B68AB4207D9284600F013
:100BF000C5FF013040F068810435F3E70025234B41
:100C0000B8463E461D70204B5D60A7E7002E3FF4BE
:100C10005BAF0BF00B030B2B7FF456AF02201B4B8B
:100C2000187001F04DF8322000F058FFB0F10009C3
:100C3000FFF64AAF19F003077FF446AF0E4A09EBFF
:100C40000503926893423FF63FAFB9F5807F3FF7C7
:100C50003BAF124BB945019322DD4FF47A7000F09F
:100C60003DFF0390039A002AFFF62EAF039A013747
:100C7000019B03F8012BEDE700220020E023002078
:100C8000C8220020F1070008E4230020DC22002015
:100C900004220020082200200C220020E022002054
:100CA000C820FFF791FD074600283FF40DAF1F2D28
:100CB00011D8C5F120020AAB25F0030084494A454A
:100CC000184428BF4A46019200F0FEFF019AFF2116
:100CD0007F4801F01FF84FEAA903C9F387027C4956
:100CE0002846019301F01EF8064600283FF46AAF3B
:100CF000019B05EB830531E70220FFF765FD002826
:100D00003FF4E2AE00F074FF00283FF4DDAE0027B0
:100D1000B946704B9B68BB4218D91F2F11D80A9B4C
:100D200001330ED027F0030312AA134453F8203CDA
:100D300005934846042205A9043702F065FA814666
:100D4000E7E7384600F01AFF0590F2E7CDF8149077
:100D5000042105A800F0E0FE00E70023642104A8B8
:100D6000049300F0CFFE00287FF4AEAE0220FFF720
:100D70002BFD00283FF4A8AE049800F02FFF05904B
:100D8000E6E70023642104A8049300F0BBFE0028DA
:100D90007FF49AAE0220FFF717FD00283FF494AECF
:100DA000049800F01DFFEAE70220FFF70DFD002880
:100DB0003FF48AAE00F02CFFE1E70220FFF704FDCC
:100DC00000283FF481AE05A9142000F027FF074654
:100DD0000421049004A800F09FFE3946B9E73220B0
:100DE00000F07CFE071EFFF66FAEBB077FF46CAE13
:100DF000384A07EB0A03926893423FF665AE022039
:100E0000FFF7E2FC00283FF45FAE27F003075744EA
:100E1000BA453FF4A3AE50460AF1040A00F0AEFE14
:100E20000421059005A800F077FEF1E74FF47A70F1
:100E3000FFF7CAFC00283FF447AE00F0D9FE0028B7
:100E400044D00A9B01330BD008220AA9002000F0ED
:100E500069FF00283AD02022FF210AA800F05AFF9B
:100E6000FFF7BAFC1C4804F0BBF913B0BDE8F08FE3
:100E7000002E3FF429AE0BF00B030B2B7FF424AEB6
:100E80000023642105A8059300F03CFE07460028D6
:100E90007FF41AAE0220FFF797FC814600283FF44A
:100EA00013AEFFF799FC41F2883004F099F90598E8
:100EB00000F0C0FF4E463C4600F078FFB0E5064625
:100EC0004CE64FF0000AFFE5B8467BE6374679E688
:100ED000E022002000220020A0860100094A49F2F9
:100EE0006900136899B21B0C00FB013344F2506196
:100EF0001360054B186882B2000C01FB02001860F9
:100F000080B27047142200201022002000211022FD
:100F100010B5044600F0FEFE034B03CB2060616079
:100F20001868A06010BD00BF00E8F11F2DE9F04374
:100F3000224DBBB002F062F940F2ED22AB68C31A59
:100F4000934232D906AF2B4628220021A8603846AA
:100F500002F032FE05F10E0000F0D4FE0026044639
:100F60005FFA80F905F10E08F3B2F100994501F13D
:100F7000280107D908EB060308223846013602F09B
:100F80001BFEF1E7082301220534297B0C48A4B29B
:100F9000CDE902320B4B01933023CDE90474009369
:100FA00004A3D3E9002302F01FFC3BB0BDE8F083AB
:100FB000AFF3008078F6339F93CACD8D905D00200B
:100FC000043400209D5D002070B50D4614461E4679
:100FD00002F0A0FB50B9022E10D1012C0ED112A3A9
:100FE000D3E900230120C5E9002307E0282C10D015
:100FF00005D8012C09D0052C0FD0002070BD302C55
:10100000FBD10BA3D3E90023ECE70BA3D3E9002327
:10101000E8E70BA3D3E90023E4E70BA3D3E900231C
:10102000E0E700BFAFF30080401DA12026812A0B1E
:1010300078F6339F93CACD8D9E6AC421818A46EE8D
:1010400026417272DF25D7B7F017304A39059E5610
:1010500013B504460846202200212346019002F0E1
:10106000ABFD227923460198032A4FF0200128BFC7
:10107000032203F8042F022202F09EFD6279234628
:101080000198072A4FF0220128BF072203F8052FF5
:10109000032202F091FDA27923460198072A4FF01E
:1010A000250128BF072203F8062F032202F084FD42
:1010B000019804F108031022282102F07DFD382058
:1010C00002B010BD2DE9F04FADF5017D0F460021B6
:1010D00040F275120EAE804622A8219100F01AFE51
:1010E00048220021304600F015FE21AD02F086F8BE
:1010F0004FF47A72554B0DF15A09B0FBF2F01860BB
:1011000093E80700012386E807000DF15A003382B7
:10111000FFF7FCFE47F605034D49338406AB18463E
:1011200006F0A0F81F2229463064304686F83C209D
:10113000FFF78EFF12AB044601460822284602F054
:101140003BFD08220DF149032846A11804F1880A45
:1011500002F032FD0DF14A03082204F11001284685
:1011600004F5847B02F028FD13AB202204F1180162
:10117000284602F021FD14AB402204F13801284634
:1011800002F01AFD16AB082204F17801284602F09D
:1011900013FD0DF15903082204F18001284602F0E5
:1011A0000BFD51460AF1080A4B460822284609F170
:1011B000010902F001FDD345F3D104F588744FF025
:1011C00000091BAB08225946284602F0F5FC96F8A8
:1011D00034304B450AD9B36B2146082228464B448C
:1011E000083409F1010902F0E7FCF0E74FF00009CB
:1011F00096F83C3004EBC9014B4508D9336C082202
:1012000028464B4409F1010902F0D6FCF0E700231F
:10121000073140460393C1F3CF01BB7E029307F130
:10122000190301930123CDE904510093F97E05A32D
:10123000D3E9002302F0D8FA0DF5017DBDE8F08F67
:10124000AFF300809E6AC421818A46EEEC23002021
:1012500094720008F8B50E4C02260E4FA4F5805388
:1012600043F8307C237E3BB965692DB1284601F0F7
:1012700041FE284605F060FF2046A4F5A55401F084
:1012800039FE012EA4F1100400D1F8BD0126E5E7D6
:1012900010590020C4730008014B1870704700BF3C
:1012A000F8230020334BF0B51C7B85B034B1324BB2
:1012B0000E221A810024204605B0F0BD2F4A02AB51
:1012C0001068516803C308232D492E480DEB030213
:1012D00005F05AFF054630B9274B0A222A481A81E1
:1012E00001F090FDE6E70169B1F5F01F06D9224B48
:1012F0000B2226481A8101F085FDDCE7438BB3F50C
:10130000AF6F09D01C4A0C21214811814FF4AF6204
:10131000194601F077FDCEE71E4A024402F11003A0
:10132000994204D2144B10221B481A81E3E710396A
:1013300020468E1A134901F067FF05F11801074690
:101340003246204601F060FFAB689F4202D1EB6855
:1013500098420AD0084B0D221A813B4600900F4854
:10136000D5E9021201F04EFDA4E70D48012401F079
:1013700049FDA0E7905D0020EC23002045730008A4
:10138000DCFF1D0000000208B4720008C0720008F3
:10139000D27200080800FEF7F07200080D73000812
:1013A000367300082DE9F04FADB080460C4606AF0D
:1013B00002F0B0F90546002859D1237E022B1BD13B
:1013C000E38A012B18D101F019FF0646FFF786FDCD
:1013D00003464FF4C87006F51676DFF8CC92B3FBDF
:1013E000F0F202FB103316FA83F3C9F80030E37E03
:1013F00033B9A84B00221A709C37BD46BDE8F08F68
:10140000A38AEEB20135013BB3420BD93B1DE90083
:10141000082220461E4401F0F8010023009602F045
:101420008FFAEDE707F11400FFF770FD324607F180
:101430001401381D05F098FE0028DAD10F2E08D8C7
:10144000944B1E70D9F80030A3F51673C9F800301C
:10145000D2E7FB1CF87001460722009303462046A2
:1014600002F06EFAF978404602F04CF9C4E7E38ADC
:10147000282B26D010D8012B1ED0052BBCD1BFF3B2
:101480004F8F8549854BCA6802F4E0621343CB60F5
:10149000BFF34F8F00BFFDE7302BADD1637EE94630
:1014A0007F4D01336A7BDBB2934203D1E27E2B7B1B
:1014B0009A4265D0CD469FE721464046FFF702FE9F
:1014C0009AE7A38A013B9BB2C92B95D8744D2E7B1A
:1014D00026BB05F10C030822314600933346204613
:1014E00002F02EFA731CF2B2D9001E46A38A013B09
:1014F0009A4205DA0E3200232A4400920822EEE7CF
:1015000000230022C5E900230023AB6085F8D73013
:10151000C5F8D8302B7B0BB9E37E2B73002507F180
:1015200014093B1D082229464846FD60C7E90155BC
:1015300002F042FB3B7A05F1010AAB424FEACA06D0
:1015400008D9FB680822314648462B44554602F02C
:1015500033FBEFE7C6F3CF060023E17E1934039394
:101560004046CDE9049663780194029328230093C2
:1015700046A3D3E9002302F037F9FFF7D7FC3BE796
:101580004FF0000807F1140310222046A7F814803A
:1015900041460093012302F0D3F9A68A023EB6B277
:1015A000F31C9B109B000733DB08A9EBC3039D468C
:1015B0000DF1180A1FFA88F34FEAC801B34201F18E
:1015C00010010AD20AEB08030822204608F101089C
:1015D0000093002302F0B4F9ECE795F8D70000F08F
:1015E000DBFAD5F8D83004461BB995F8D70000F0DF
:1015F000E3FAD5F8D83033449C4204D295F8D700AA
:10160000013000F0D9FA4FEA960B4FF000081FFAAC
:1016100088F18B45D5E9003209D90AEB880101220E
:1016200003EB880008F1010800F07CFBEFE7F318FA
:1016300095F8D70042F10002C5E90032D5F8D8305C
:1016400006EB0308C5F8D88000F0A6FA804509D358
:1016500095F8D730D5F8D8000133001B85F8D7307E
:10166000C5F8D800FF2E08D800232B7300F0C0FA6D
:10167000FFF718FE08B1FFF7EDF82B68094A9B0A3F
:10168000013313810023AB6014E700BF264172725F
:10169000DF25D7B7FD33002000ED00E00400FA0598
:1016A000905D0020EC2300200034002010B54FF0A6
:1016B00040540C4B22689A4212D1627D0A4B0B486F
:1016C0001A70C922237D0E30094900F8023C00F04F
:1016D000FBFAE0220021204600F01CFB012010BD97
:1016E0000020FCE79AAD44C5F8230020905D00205F
:1016F0001600003037B502231D4C1E4D0122204636
:101700001D496B71236804F580545B689847D4F8D1
:10171000B034012218495B6804F5966098470023AD
:1017200016494FF480520193154B16480093164BFF
:1017300001F0C2FF154B197811B1124801F0E2FF18
:1017400001F05CFD0446FFF7C9FB4FF4C873B0FB22
:10175000F3F202FB130304F5167010FA83F00C4B3E
:10176000186004F0E1F908B10F232B8103B030BDFC
:1017700030340020EC23002040420F00FC230020E6
:10178000C90F000804340020A5130008F823002026
:10179000003400202DE9F04F9C4D2DED028B93B0CD
:1017A000DFF890A29A4F284602F082F803460028FC
:1017B0003DD00024974E0E94A046ADF84440A1467B
:1017C000CDE90F44027B8DF844200FAA9968406848
:1017D00003C21B6843F000430E93336804F22C5499
:1017E000D3F810B001F00CFD10EB0A02CDF8009018
:1017F000304606F5A55641F100030EA9D84740F63C
:1018000058230028C8BF48F0010810369C42E4D194
:10181000B8F1000F05D0284602F04EF887F8009086
:10182000C1E73B78072B00F2E08001333B700023D7
:101830000DF12C084FF0010A0A93ADF834300B93E8
:10184000C8F804309FED6B8B0026724C3746236836
:101850004FF0000B0DF11D0207A920468DF81CA0CA
:101860008DF81DB08DED008BD3F808905B46C8470E
:101870009DF81C90B9F1000F1ED0102259460EA8F9
:1018800000F048FA236808AA0AA95F6920460DF10A
:101890001E03B8470FAB4F4698E8030083E80300E8
:1018A0009DF834300EA928468DF844300A9B0E93DB
:1018B000DDE9082302F0C8F906F22C5640F6582359
:1018C00004F5A5549E4204F11004C0D1002FBBD1F1
:1018D000284601F01FFF002840D14F4E01F08EFC3A
:1018E000336898423AD301F089FC0446FFF7F6FAD0
:1018F0004FF4C87304F516748DF82870B0FBF3F23A
:1019000002FB130314FA83F33360444E377817B99C
:1019100001238DF82830C7F110040EA8FFF7F6FA5E
:101920000EABE4B20DF12900D919062C28BF06240C
:101930002246013400F0C8F90AABE4B2284603930A
:10194000182304940293364B0193012300932BA395
:10195000D3E9002301F0E0FE0023337001F04EFCD8
:10196000304A314C1368C31AB3F57A7F30D3106014
:1019700001F046FC02460B46284601F0A7FF284628
:1019800001F0C8FE20B3237B0EAF284E002B14BFFE
:1019900003230223737101F031FC4FF47A7339464B
:1019A000B0FBF3F030603046FFF752FB18230730EE
:1019B00002931F4BC0F3CF00019340F25513CDE9C2
:1019C0000370009328460FA3D3E9002301F0A4FE7F
:1019D000237B2BB1FFF7AAFA237B002B7FF4E0AE29
:1019E00013B0BDEC028BBDE8F08F284601F064FF18
:1019F0001DE700BF0000000000000000401DA12006
:101A000026812A0BF1C6A7C1D068080F0434002034
:101A1000755E00203034002000340020FD330020AB
:101A2000FC330020705E0020905D0020EC2300203D
:101A3000745E002040420F0008B5064800F014FD17
:101A4000054800F011FD054A05490020BDE80840A1
:101A500005F06CBB30340020E0480020D05E002050
:101A600055120008F7B50C46184E4FF47A7105462A
:101A700002FB01F396F90020501C0BD114482946B3
:101A800001930268176A2246B8478442019B03D13A
:101A9000002310E0002AF1D096F90020511C01D05B
:101AA000012A0DD10B4829460268166A2246B04722
:101AB000844205D10123084A0120137003B0F0BD10
:101AC0004FF4FA7003F08CFB0020F7E71822002097
:101AD000F8640020D45E0020BC5E0020002307B51F
:101AE000024601210DF107008DF80730FFF7BAFF1C
:101AF00020B19DF8070003B05DF804FB4FF0FF3004
:101B0000F9E700000A46042108B5FFF7ABFF80F0B3
:101B10000100C0B2404208BD074B0A4630B41978F4
:101B2000064B53F82140014623682046DD69044BEB
:101B3000AC4630BC604700BFBC5E00206C73000840
:101B4000A086010070B50A4E00240A4D03F0F4FD92
:101B5000308028683388834208D903F0E9FD2B6878
:101B600004440133B4F5003F2B60F2D370BD00BFD5
:101B7000BE5E0020785E002003F0BCBE00F1006075
:101B800000F500300068704700F10060920000F539
:101B9000003003F033BE0000054B1A68054B1B886C
:101BA0009B1A834202D9104403F0C2BD0020704743
:101BB000785E0020BE5E002038B5074D04462868D8
:101BC000204403F0BBFD28B928682044BDE8384014
:101BD00003F0C6BD38BD00BF785E0020002070470E
:101BE00000F1FF5000F58F10D0F80008704700009A
:101BF000064991F8243033B100230822086A81F89D
:101C00002430FFF7C1BF0120704700BF7C5E002079
:101C1000014B1868704700BF0010005C244BF0B502
:101C20001A680446234BC2F30B06120C1F8858682F
:101C3000BE4293F9085028D09F89BE4206D10120A8
:101C40000C2505FB0033586893F9085041F2010355
:101C50009A421CD041F203039A421AD042F2010385
:101C60009A4218D042F203039A4208BF5625621ED8
:101C70000B46441E0A4493420FD214F9016F581CBC
:101C80006EB1034600F8016CF5E70020D8E75A254D
:101C9000EDE75925EBE75825E9E7184605E02C2440
:101CA00082421C7001D9981C5D70401AF0BD00BFC3
:101CB0000010005C1C2200200020704770470000CC
:101CC0007047000070470000002310B5934203D016
:101CD000CC5CC4540133F9E710BD0000013810B5E5
:101CE00010F9013F3BB191F900409C4203D11AB178
:101CF0000131013AF4E71AB191F90020981A10BDA8
:101D00001046FCE703460246D01A12F9011B0029CF
:101D1000FAD1704702440346934202D003F8011BF4
:101D2000FAE770472DE9F8431F4D144607468846E9
:101D300095F8242052BBDFF870909CB395F82430BE
:101D40002BB92022FF2148462F62FFF7E3FF95F8C9
:101D500024004146C0F1080205EB8000A24228BFE2
:101D60002246D6B29200FFF7AFFF95F82430A41BAD
:101D700017441E449044E4B2F6B2082E85F824605D
:101D8000DBD1FFF735FF0028D7D108E02B6A03EB42
:101D900082038342CFD0FFF72BFF0028CBD1002056
:101DA000BDE8F8830120FBE77C5E0020024B1A7837
:101DB000024B1A70704700BFBC5E00201822002042
:101DC00038B5164C164D204602F000FD2946204637
:101DD00002F028FD2D681348D5F89020D2F8043879
:101DE00043F00203C2F8043803F0FAF90E4928461A
:101DF00002F026FED5F890200C48D2F804380C49A1
:101E0000A04223F00203C2F804384FF4E1330B6020
:101E100003D0BDE8384002F037BC38BDF86400207C
:101E20000C75000840420F0014750008D45E0020B5
:101E3000A45E002038B50B4B04461A780A4B53F8C1
:101E400022500A4B9D420CD0094B00211822184603
:101E5000FFF760FF046001462846BDE8384002F005
:101E600013BC38BDBC5E00206C730008F864002011
:101E7000A45E0020202383F3118862B6704700001F
:101E8000002383F3118862B6704700000120704779
:101E9000704700007047000010B4134602681468D1
:101EA0000022A4465DF8044B6047000000F5805016
:101EB00090F859047047000000F5805090F85204E3
:101EC0007047000000F5805090F9580470470000FA
:101ED0004E20704700F5805208B5FFF7CBFFD2F8CF
:101EE0009834D2F894041844D2F890341844D2F8B4
:101EF00078341844D2F888341844D2F8843418441A
:101F0000FFF7BEFF08BD00002DE9F74F0C4600F5B6
:101F100080511F46054691F852349046BDF83090E6
:101F20009BB1D1F874340133C1F8743423689A003A
:101F300006D4237B082B0BD9627B0AB10F2B07D960
:101F4000D1F878340133C1F878344FF0FF300FE026
:101F5000FFF790FFEB6AD3F8C42012F4001A0AD0FE
:101F6000D1F87C3400200133C1F87C34FFF788FFBE
:101F700003B0BDE8F08F22684FF0480BD3F8C4607F
:101F8000002A6B6AC6F30446B4BF42F08042920452
:101F90001BFB063BCBF8002023685B004FEA06637F
:101FA00044BF42F00052CBF80020227B43EA0243B8
:101FB0007201CBF80430607B18B343F44013CBF8C4
:101FC0000430D1F8A4340133C1F8A434AB1803F5BC
:101FD0008353197B41F020011973207B019200F09B
:101FE0006DFF0330019A80105FFA8AF30AF1010A4B
:101FF00083420DDA04EB83010BEB8303496899609C
:10200000F2E7AB1803F58353197B60F34511E3E75F
:102010000121EB6A04F10C00B140C3F8D010AB18F9
:10202000214603F58253C3E9048705EB461303F504
:102030008253183351F804CB814243F804CBF9D1D1
:1020400009882A442846198041F26803D65002F5CF
:10205000805209F0030392F86C1043F0100321F052
:102060001F010B43214682F86C304246FFF708FF00
:102070003B46CDF8309003B0BDE8F04F00F0E4BE31
:102080002DE9F04700F58056044696F85254002D8D
:1020900040F00181037C032B40F092802B462846C0
:1020A0002F465FFA83FC944510DA01EBCC0E51F811
:1020B0003CC0BCF1000F04DBDEF804C0BCF1000F33
:1020C00002DB01370133ECE70130FBE7FFF7D2FE1B
:1020D000E36AF0B9D3F8800040F00200C3F8800052
:1020E0004E23E06A002F6ED1D0F8803043F0010318
:1020F000C0F88030694B6A4A1B6803F1805303F5CE
:102100002C539B009342A36240F2AF80654801F0DC
:102110006FF84D2842D8DFF884814FEA004EDFF88F
:102120008891D8F800C04EEA8C0EC3F884E00CF118
:10213000805303F52C539B00636100EB0C03D4F830
:102140002CC0C8F80030C0F14E03DCF8800040F02D
:102150003000CCF880004FF0000CD4F81480E64634
:102160005FFA8CF08242BCDD01EBC00A51F830000E
:10217000002810DBDAF804A0BAF1000F0BDA09EA44
:1021800000400AF07F0A40EA0A0040F0084048F8A0
:102190002E000EF1010E0CF1010CE1E79A6922F01C
:1021A00001029A6101F02AF80646E36A9B69D907A1
:1021B00004D501F023F8831BFA2BF6D9FFF760FE54
:1021C0002846BDE8F087B7EB530F3DD2DFF8CCE0EF
:1021D0004FEA074CDEF800304CEA830CC0F888C0A8
:1021E00003F1805003EB4703002700F52C50CEF895
:1021F0000030BC468000A061E06AD0F8803043F037
:102200000C03C0F88030D4F818E0FBB29A427FF794
:1022100071AF51F8330001EBC3080028D8F804303F
:1022200001DB002B0EDB20F0604023F0604340F028
:10223000005043F000434EF83C000EEBCC000CF194
:10224000010C43600137E0E7836923F001038361F8
:1022500000F0D4FF0646E36A9B69DA07AED500F0CA
:10226000CDFF831BFA2BF6D9A8E7E26A936923F026
:102270000103936100F0C2FF0746E36A9B69DB0735
:1022800005D500F0BBFFC31BFA2BF6D996E7012555
:1022900086F8525492E7002592E700BFCC5E0020FA
:1022A000FCB50040747300080000FF0713B500F58B
:1022B00080540191606C00F053FE1F280AD920223F
:1022C0000199606C00F0C2FEA0F120035842584111
:1022D00002B010BD0020FBE700F5805008B5FFF705
:1022E000C9FD406C00F010FEBDE80840FFF7C8BD16
:1022F00000220260828142608260704700220023D7
:1023000010B5C0E90023002304460C3020F8043C3B
:10231000FFF7EEFF204610BD2DE9F047074688B0D5
:102320009A46884607F5805468469146FFF7A2FD15
:10233000FFF7E4FF606C00F0F9FD1F282DD9202283
:102340006946606C00F006FF202826D194F85234CC
:102350001BB303AD444605AB2E46083403CE9E4264
:1023600044F8080C44F8041C3546F5D13068414661
:1023700020603846B388A380DDE90023C9E9002343
:10238000BDF808304A46AAF80030FFF779FD5346F9
:1023900008B0BDE8F04700F045BD0020FFF770FD34
:1023A00008B0BDE8F08700002DE9F84F002306468D
:1023B00000F58154054688461034C0E90133274BA7
:1023C00046F8303B374638462037FFF797FFA7429D
:1023D000F9D105F580544FF4805305F5A3594FF01A
:1023E000000A26630026676405F5835709F1100982
:1023F0004FF0000B1037E663C4E90D36012384F873
:10240000403084F84830A7F11800203747E910AB76
:10241000FFF76EFF47F8286C4F45F4D1B8F1010F74
:1024200084F85884A4F85A64A4F85C64A4F85E6440
:1024300084F86064A4F86264A4F86464A4F8666430
:1024400084F8686402D9064800F0D2FE054B28469D
:1024500053F82830EB62BDE8F88F00BFC473000862
:1024600098730008B4730008044B10B5197804463B
:102470004A1C1A70FFF798FF204610BDC95E002065
:102480002DE9F04700295FD0304F3148B7FBF1F517
:1024900081428CBF0A201120431EB5FBF0FC00FBDB
:1024A0001C50DCB220B1022B1846F5D8002037E0D2
:1024B0000CF1FF35B5F5806F32D2C4EBC4094FF48F
:1024C0007A7009F103034FEAE308C3F3C70308F185
:1024D000010AA4EB030E08FB00085FFA8EF65AFA15
:1024E0008EFEB8FBFEFEBEF5617F1BDC1FFA8EF48C
:1024F000581C56FA80F00CFB00FCB7FBFCFC614555
:10250000D4D1013BDBB20F2BD0D8711E0020C9B251
:10251000072905D8107101201480558053719171DD
:10252000BDE8F08709F1FF334FEAE30EC3F3C703B9
:102530000EF10108E41A0EFB0000E6B258FA84F42A
:10254000B0FBF4F4A4B2D3E70846E9E700B4C4044E
:102550003F420F0038B540F27772C36A154CC3F89A
:10256000BC200722C36AC3F8C8202268C16A93004E
:1025700043F4C023C1F8A03002F1805302F16C0192
:10258000C56A03F52C53EA3289009B00226041F0B2
:10259000E061094AC361C5F8C01003F5D87103F5BD
:1025A0006A7341629342836202D9044800F020FEBC
:1025B00038BD00BFCC5E0020FCB50040747300083D
:1025C0002DE9F04F00F58055994689B0044695F8FD
:1025D00058348A469046022B04D90027384609B061
:1025E000BDE8F08F9E4A52F8231009B942F8230043
:1025F0009C49C4F80CA00B7884F81090C3B9FFF77D
:1026000039FC994BD3F8EC2042F48072C3F8EC20EB
:10261000D3F8942042F48072C3F89420D3F8942025
:1026200022F48072C3F8942001230B70FFF728FC7A
:1026300095F851346BB9FFF71DFC8C4A95F8583466
:10264000D35CEBB1012B24D0012385F85134FFF783
:1026500017FCFFF70FFCE26A936923F01003936104
:1026600000F0CCFD0746E36A9E6916F0080617D015
:1026700000F0C4FDC31BFA2BF5D9FFF701FCACE752
:102680000221132001F04EFE0221152001F04AFE26
:10269000DAE70221142001F045FE02211620F5E7B9
:1026A0009A6942F001029A6100F0A8FD0746E36AC8
:1026B0009A69D00705D400F0A1FDC31BFA2BF6D907
:1026C000DBE79A69002704F5825B42F002020BF116
:1026D000100B9A61E36A5F65FFF7D2FB686C00F04C
:1026E00013FC202200216846FFF714FB02A8FFF725
:1026F000FFFD6A460BEB06030DF1180E0697944694
:102700000833BCE80300F44543F8080C43F8041C04
:102710006246F4D1DCF8000020361860B6F5806F10
:102720009CF804201A71DCD1002304F5A252514612
:1027300020461A3285F8503485F85334FFF7A0FE4E
:10274000074690B9E26A936923F00103936100F0B0
:1027500055FD0546E36A9B69D9077FF53EAF00F05A
:102760004DFD431BFA2BF5D937E795F85F6495F8D3
:102770005E243602C5F86CA4E36A46EA426695F820
:1027800060241643B5F85C2446EA0246DE61B8F1DF
:10279000000F29D004F5A352414620460232FFF72C
:1027A0006FFE90B9E26A936923F00103936100F030
:1027B00025FD0546E36A9B69DA077FF50EAF00F059
:1027C0001DFD431BFA2BF5D907E795F8683495F8FA
:1027D00067141B01C5F87084E26A43EA0123B5F867
:1027E000641443EA0143D360E36A00262046C3F839
:1027F000BC60FFF7AFFE85F859646FF04042E36AB2
:10280000B9F1030F1A651A4AE36A5A654FF00222BA
:10281000E36A9A654FF0FF32E36AC3F8E0204FF0B5
:102820000302E36ADA65E26A936943F440739361F1
:102830003FF4D4AEE26A936923F00103936100F0A0
:10284000DDFC0646E36A9B69DB0705D500F0D6FC94
:10285000831BFA2BF6D9C0E6012385F85234BDE676
:10286000C05E0020C85E002000440258AC7300081F
:10287000550200022DE9F04F054689B09046994671
:10288000002741F2680A00F58056EB6AD3F8D83089
:10289000FB40D8074AD505EB47124FEA471B524485
:1028A0001379190742D4D6F880340133C6F880343E
:1028B00013799A0605EB0B0248BFD6F8A8345244A8
:1028C00044BF0133C6F8A834137943F008031371E9
:1028D000DB0723D596F8533403B305F582546846D5
:1028E000FFF70CFD03AB18345C4404F1080C2068BE
:1028F000083454F8041C1A46644503C21346F6D142
:102900002068694610602846A2889A800123ADF8A5
:1029100008302B68CDE900891B6C9847D6F85434F1
:1029200023B1D6F89C340133C6F89C340137202FEC
:10293000ABD109B0BDE8F08F2DE9F04F0F468DB057
:10294000044600F05DFC82468946002F5BD1E36AB5
:10295000D3F8A02012F4FE0F03D100200DB0BDE883
:10296000F08FD3F8A420920141BF04F58051D1F833
:1029700094240132C1F89424D3F8A4205606ECD054
:10298000D3F8A450E669C5F305254823E8464FF07F
:10299000000B03FB05664046FFF7AAFC32685100B6
:1029A0004ABF22F06043C2F38A4343F000439200DF
:1029B00048BF43F080430093736813F400131BBFB8
:1029C000012304F580528DF80D308DF80D301EBFB7
:1029D000D2F8AC340133C2F8AC34F38803F00F03FF
:1029E0008DF80C309DF80C0000F068FA5FFA8BF35C
:1029F000984225D9F2180CA90BF1010B127A0B445D
:102A000003F82C2CEEE7012FA7D1E36AD3F8B0200E
:102A100012F4FE0FA1D0D3F8B420950141BF04F504
:102A20008051D1F894240132C1F89424D3F8B42011
:102A3000500692D0D3F8B450266AC5F30525A4E712
:102A4000EFB9E36AC3F8A85004A807ADFFF756FC36
:102A500098E80F0007C52B800023204604A9ADF895
:102A60001830236804F580541B6CCDE904A99847FD
:102A700058B1D4F88C340133C4F88C346EE7012F8C
:102A8000E2D1E36AC3F8B850DEE7D4F8903401200D
:102A90000133C4F8903461E7F8B505460F4600F5F8
:102AA0008054012639462846FFF746FF10B184F8C6
:102AB0005364F7E7D4F8543423B1D4F89C34013389
:102AC000C4F89C34F8BD0000C36AF0B51A6C12F467
:102AD0007F0F2BD01B6C00F5805441F268054FF03E
:102AE000010CC4F8A0340023471900EB43125E0127
:102AF0002A44117911F0020F15D0490713D4B9599E
:102B0000C66A0CFA01F1D6F8CCE011EA0E0F0AD031
:102B1000C6F8D410117941F004011171D4F8882459
:102B20000132C4F888240133202BDED1F0BD00002F
:102B30002B4B70B51E561B5C012B30D8294D2A4AF1
:102B400055F8233052F8264013B349B3236D9A0544
:102B500010D54FF40073236500F052FB50EA0102D8
:102B60000B4602D0013861F10003024655F82600F9
:102B7000FFF780FE236D9B012CD54FF0007255F8B6
:102B80002630226503F58053012283F8592421E081
:102B900001232365102323654FF48053236570BD03
:102BA000236DDA0702D4236D5B0706D505230021C8
:102BB00055F826002365FFF76FFF236DD80602D472
:102BC000236D590606D55023012155F826002365AB
:102BD000FFF762FF55F82600BDE87040FFF774BFAD
:102BE000B0730008C05E0020B473000808B5FFF79A
:102BF00041F9FFF769FFBDE80840FFF741B9000060
:102C0000C36AD3F8C00010F07C5005D0D3F8C400DC
:102C100080F40010C0F340507047000000F5805071
:102C200008B5FFF727F9406C00F080F9FFF728F9A5
:102C300043090CBF0120002008BD000000F58053AF
:102C400093F8592462B1C16A8A6922F001028A614B
:102C5000D3F898240132C3F89824002283F8592429
:102C6000704700002DE9F74300F582519846002592
:102C7000FFF700F9103141F2680E4FF0010900F53D
:102C8000805C00EB4514744423795E071CD4DB069A
:102C90001AD58E69C36A09FA06F6D3F8CC703E429B
:102CA00012D04F6801970F689742019F77EB080792
:102CB0000AD2C3F8D460237943F004032371DCF80B
:102CC00084340133CCF8843401352031202DD8D11F
:102CD00003B0BDE8F043FFF7D3B80000F8B51E46D7
:102CE00000230F46054613701446FFF797FF80F048
:102CF000010038701EB12846FFF782FF2070F8BD32
:102D00002DE9F04F994685B00B780E468046174660
:102D100001931378DDE90EBA029300F071FA33786B
:102D200004460D4613B93B78002B41D022462B4672
:102D30004046FFF797FFFFF759FFFFF77FFF4B462E
:102D40003A463146FFF7CAFF33782BB1019B1BB1DE
:102D5000012005B0BDE8F08F3B7813B1029B002B3A
:102D6000F6D108F5805303935C4575EB0A031FD237
:102D7000039BD3F85404D8B1BBEB04020368D968B1
:102D80006AEB050388474B463A4631464046FFF713
:102D9000A5FF337813B1019B002BD9D13B7813B138
:102DA000029B002BD4D100F02BFA04460D46DBE742
:102DB0000020CEE7002108B50846FFF7B9FEBDE8C0
:102DC000084001F075B9000008B501210020FFF7A7
:102DD000AFFEBDE8084001F06BB9000008B5002166
:102DE0000120FFF7A5FEBDE8084001F061B9000031
:102DF000012108B50846FFF79BFEBDE8084001F039
:102E000057B900000FB4002004B0704713B56C46EA
:102E1000031D84E8060094E8030083E80500012010
:102E200002B010BD73B58568019155B11B885B0771
:102E300007D4D0E90036DB6B9847019AC1B230461F
:102E4000A847012002B070BDF0B5866889B005467C
:102E50000C465EB1BDF838305B070AD4D0E90037C4
:102E6000DB6B98472246C1B23846B047012009B013
:102E7000F0BD0022002301F10806CDE90023002364
:102E80000A46ADF8083003AB1068083252F8041C4B
:102E90001C46B24203C42346F6D1106820609288D3
:102EA000A28000F0AFF90423ADF808302B68CDE91B
:102EB00000011B6C694628469847D7E7082817D9B0
:102EC00009280CD00A280CD00B280CD00C280CD0C8
:102ED0000D280CD00E2814BF4020302070470C2045
:102EE000704710207047142070471820704720202A
:102EF0007047000010B5037C044613B9006804F065
:102F00002BF9204610BD00000023BFF35B8FC36088
:102F1000BFF35B8FBFF35B8F8360BFF35B8F704743
:102F2000BFF35B8F0068BFF35B8F704770B50546DA
:102F30000C30FFF7F5FF044605F108063046FFF7B1
:102F4000EFFFA04206D96D683046FFF7E9FF254440
:102F5000281A70BD3046FFF7E3FF201AF9E700009A
:102F600070B505464068A0B105F10C0605F10800F2
:102F7000FFF7D6FF04463046FFF7D2FF844204F144
:102F8000FF34304694BF6D680025FFF7C9FF2C441D
:102F9000201A70BD38B50C460546FFF7C7FFA042A2
:102FA00010D305F10800FFF7BBFF04446868BFF3C6
:102FB0005B8FB4FBF0F100FB11440120AC60BFF368
:102FC0005B8F38BD0020FCE72DE9F0411446074631
:102FD0000D46FFF7C5FF844228BF0446D4B1B8466A
:102FE00058F80C6B4046FFF79BFF30442860404682
:102FF0007E68FFF795FF331A9C4203D801206C606E
:10300000BDE8F081A41B6B603B682044AB60E860C6
:103010000220F5E72046F3E738B50C460546FFF7F2
:103020009FFFA04210D305F10C00FFF779FF044485
:103030006868BFF35B8FB4FBF0F100FB1144012023
:10304000EC60BFF35B8F38BD0020FCE72DE9FF414A
:103050008846694607466C46FFF7B6FF002506B26C
:1030600004EBC606B4420AD0626808EB050120688A
:103070000834FEF729FE54F8043C1D44F2E72946C3
:103080003846FFF7C9FF284604B0BDE8F0810000CC
:10309000F8B505460C300F46FFF742FF05F108066C
:1030A00004463046FFF73CFFA042304688BF6C68BC
:1030B000FFF736FF201A386020B12C683046FFF742
:1030C0002FFF2044F8BD000073B5144606460D4698
:1030D000FFF72CFF8442019028BF0446DCB101A910
:1030E0003046FFF7D5FF019B33B93268C5E902339B
:1030F000C5E9002401200CE09C42286038BF0194FF
:10310000019884426860F5D93368241A0220AB60C4
:10311000EC6002B070BD2046FBE700002DE9FF41E6
:103120000F4669466C46FFF7CFFF00B2002604EB5E
:10313000C005AC4209D0D4F80480B81954F8081B73
:1031400042464644FEF7C0FDF3E7304604B0BDE812
:10315000F081000038B50546FFF7E0FF0446014660
:103160002846FFF717FF204638BD000000B59BB08A
:10317000EFF3098168226846FEF7A6FDEFF30583A9
:10318000044B9A6BDA6A9A6A9A6A9A6A9A6A9A6A93
:103190009B6AFEE700ED00E000B59BB0EFF309810C
:1031A00068226846FEF790FDEFF30583044B9A6BA7
:1031B0009A6A9A6A9A6A9A6A9A6A9B6AFEE700BF52
:1031C00000ED00E000B59BB0EFF30981682268468E
:1031D000FEF77AFDEFF30583034B5A6B9A6A9A6AFE
:1031E0009A6A9A6A9B6AFEE700ED00E0FEE700003B
:1031F0000FB408B5029801F083FFFEE702F0C2BBEE
:1032000002F09ABB02F098BB30B50A44084D9142D7
:103210000DD011F8013B5840082340F30004013B56
:103220002C4013F0FF0384EA5000F6D1EFE730BDE5
:103230002083B8ED2DE9F041C56915B9C161BDE83C
:10324000F0814B68AC4623F06047C3F38A464FEAEF
:10325000D37EC3F3807816EA230638BF3E462B465A
:103260005A68BEEBD27F22F060440AD0002A18DAF6
:10327000A40CB44217D19D420FD10D60DEE7134676
:10328000EEE7A74207D102F08044C2F380724245C4
:103290000BD054B1EFE708D2EDE7CCF800100B608B
:1032A000CDE7B44201D0B442E5D81A689C46002A62
:1032B000E5D11960C3E700002DE9F047089D01F052
:1032C000070400EBD1004FF47F494FEAD5082244B0
:1032D00005F00705944201D1BDE8F08704F0070727
:1032E00005F0070A111B08EBD50E57453E4613F8AB
:1032F0000EC038BF5646C6F108068E4228BF0E469D
:10330000E108415C34443544B94029FA06F721FA12
:103310000AF1FFB28CEA010147FA0AF739408CEA58
:10332000010C03F80EC0D5E780EA0120082341F222
:10333000210201B2013B4000002980B2B8BF5040D9
:1033400013F0FF03F5D1704738B50C468D18A54230
:1033500000D138BD14F8011BFFF7E6FFF7E70000C6
:1033600002684AB1136801890360C38801339BB2C4
:103370009942C38038BF03811046704770B588B04A
:10338000044620220D4668460021FEF7C3FC204675
:103390000495FFF7E5FF024660B16B46054608AEAF
:1033A0001C46083503CCB44245F8080C45F8041C0B
:1033B0002346F5D1104608B070BD0000082817D983
:1033C00009280CD00A280CD00B280CD00C280CD0C3
:1033D0000D280CD00E2814BF4020302070470C2040
:1033E0007047102070471420704718207047202025
:1033F00070470000082817D90C280CD910280CD9C0
:1034000014280CD918280CD920280CD930288CBFA6
:103410000F200E207047092070470A2070470B20AC
:1034200070470C2070470D207047000010B54B68A6
:1034300023B9CA8A63F30902CA8210BDC4681A6834
:103440001C60C360438A013B43824A60EFE700008F
:103450002DE9F84F1D46CB8A0F468146C3F309017B
:10346000924606290B4630D00020AAB207F1190473
:103470009EB21FFA80F8052E0FD8904503F1010384
:1034800006D30A44FB8A62F309030120FB821AE097
:103490001AF800600130E654EAE79045F1D2A1F154
:1034A000060B1C237C68BBFBF3F203FB12BB1FFA69
:1034B0008BF6002C45D14846FFF752FF044638B939
:1034C00078606FF00200BDE8F88F4FF00008E6E783
:1034D000002606607860ADB24FF0000B454510D96C
:1034E0000AEB0803221D13F8011B08F1010891558E
:1034F000B1B21FFA88F81B292BD0454506F1010609
:10350000F1D8FB8AC3F30902154465F30903BCE74C
:1035100001321C4692B22368002BF9D1AB1F0B4439
:103520001C21B3FBF1F301339BB29A42D3D2BBF11E
:10353000000FD0D14846FFF713FF20B9C4F800B000
:10354000BFE70122E7E7C0F800B05E46206004460E
:10355000C1E74545D5D94846FFF702FF08B92060C5
:10356000AFE7C0F800B0002620600446B6E70000D0
:103570002DE9F04F2DED028B83B007469146BDF843
:103580003C50CDE90013002A00F092802DB10E9B33
:10359000002B00F08D80072D32D807F10C00FFF7CB
:1035A000DFFE044638B96FF00204204603B0BDECDC
:1035B000028BBDE8F08F14220021FEF7ABFB2A46F8
:1035C0000E9904F10800FEF77FFB681CC0B2FFF7FC
:1035D00011FFFFF7F3FE207499F80030013803F073
:1035E0001F0314FA80F063F03F0303723846009B18
:1035F00043F0004161602146FFF71CFE0124D4E73F
:103600004FF0000800F10C034FF0800A4646444694
:1036100008EE103A18EE100AFFF7A2FE83460028C3
:10362000C1D014220021FEF775FBC6BB019B02200E
:10363000ABF808300E9B00F1080299195BFA82F290
:103640000130C0B2082801D0AE422AD3FFF7D2FE23
:10365000AE4208BF4FF0400AFFF7B0FE99F80020D5
:10366000411E009B02F01F0201345BFA81F142EA25
:10367000481288F0010824B24AEA020A43F00042E4
:1036800081F808A059468BF810003846CBF8042082
:103690004FF0000AFFF7CEFDAE42BBD185E7002018
:1036A000C8E711F801CB013602F801CBB6B2C7E783
:1036B0006FF0010479E70000F8B515460E462822A0
:1036C000002104461F46FEF725FB069BB5F5001FAB
:1036D000A760636004F10C00079B34BF6A094FF6D2
:1036E000FF722362002397B29A4205D80023036039
:1036F00027826382A382F8BD0660013330462036FC
:10370000F2E7000003781BB94BB2002BC8BF017071
:1037100070470000007870472DE9F74FDDF83C90C6
:10372000804692469B46BDF830500D9E9DF838402D
:10373000BDF84070B9F1000F01D1002F51D11F2CFD
:103740004FD898F80000B0B9072F47D835F00303D9
:1037500047D13A4649464FF6FF702D02FFF7F4FD78
:1037600020F0010045EA04644004400C44EA40248F
:103770004FF6FF7321E040EA0520072F40EA04647A
:10378000F6D900254FF6FF73C5F12000A5F1200200
:103790002AFA05F108350BFA00F02BFA02F2014380
:1037A00018461143C9B2FFF7BFFD402D0346EBD1C8
:1037B0003A464946FFF7C8FD034632462146404691
:1037C000CDE90097FFF7D4FE33780133DBB21F2B2E
:1037D00088BF0023337003B0BDE8F08F6FF00300A3
:1037E000F9E76FF00100F6E72DE9F04F85B092465A
:1037F00006469B46DDF848800F9D9DF840209DF8C9
:103800004490BDF84C70B8F1000F01D1002F49D1A0
:103810001F2A47D83378002B47D00C029DF8381068
:10382000072F44EA026444EAC93444EA014444EA02
:10383000030444F0800432D900234FF6FF72C3F131
:10384000200CA3F120002AFA03F103930BFA0CFCDD
:103850002BFA00F041EA0C0101431046C9B2FFF710
:1038600063FD039B02460833402BE8D13A464146AC
:10387000FFF76AFD03462A4621463046CDE9008718
:10388000FFF776FEB9F1010F06D12B780133DBB2D9
:103890001F2B88BF00232B7005B0BDE8F08F4FF6BB
:1038A000FF73E8E76FF00100F6E76FF00300F3E75E
:1038B000C06900B104307047C3691A68C261C26848
:1038C0001A60C360438A013B438270472DE9F0418F
:1038D000D0F8188014461D46184E4146002709B9F5
:1038E000BDE8F081D1E90223A21A65EB03039642F9
:1038F00077EB03031ED283698B420DD1FFF796FD50
:1039000083691B688361C3680B60438AC160013BA4
:10391000816943828846E2E7FFF788FD0B68C8F8B3
:103920000030C3680B60438AC160013B4382D8F812
:103930000010D4E788460968D1E700BF80841E00E4
:103940002DE9F04F8BB00D4614469B46DDF85090A4
:103950008046002800F01881B9F1000F00F01481B2
:10396000531E3F2B00F21081012A03D1BBF1000F3F
:1039700040F00A810023CDE90833B8F81430B5EBE4
:10398000C30F4FEAC30703D300200BB0BDE8F08F8D
:103990002B199F42D8F80C3036BF7F1B2746FFB249
:1039A0001BB9D8F81030002B7AD02F2D4DD8C5F187
:1039B000300600232946B742009308ABD8F8080028
:1039C0002CBFF6B23E46A7EB060A354432465FFAF4
:1039D0008AFAFFF771FCB8F81430302103F1005374
:1039E000063BDB000493D8F80C300393039B13B120
:1039F000BAF1000F2CD1D8F8100040B1BAF1000F85
:103A000005D008AB5246691A0096FFF755FC38B24C
:103A1000002FB9D066070AD00AAB624203EBD4018B
:103A200002F0070211F8083C134101F8083C082C89
:103A30003DD9102C40F2B580202C40F2B780BBF16C
:103A4000000F00F09C80082335E0BA460026C2E74C
:103A5000049BE02B28BFE02306930B44AB42059365
:103A600015D95A1B0398691A0096924508AB00F1C4
:103A7000040034BF5246D2B20792FFF71DFC079AEA
:103A80001644AAEB020A1544F6B25FFA8AFA049BBE
:103A9000069A05999B1A0493039B1B680393A5E759
:103AA00000933A4608AB2946D8F80800ADE7BBF1C9
:103AB000000F13D00123B4EBC30F6BD0082C12D826
:103AC0009DF82030621E23FA02F2D50706D54FF08A
:103AD000FF3202FA04F423438DF820309DF82030A1
:103AE00089F8003051E7102C12D8BDF82030621E42
:103AF00023FA02F2D10706D54FF0FF3202FA04F49E
:103B00002343ADF82030BDF82030A9F800303CE761
:103B1000202C0FD80899631E21FA03F3DA0705D584
:103B20004FF0FF3202FA04F40C430894089BC9F8E2
:103B300000302AE7402C2AD0611EC4F12102A4F1F2
:103B40002103DDE9086526FA01F105FA02F225FAFA
:103B500003F311431943CB0711D50122A4F120032C
:103B6000C4F1200102FA03F322FA01F1A2400B434F
:103B7000524263EB430332432B43CDE90823DDE993
:103B80000823C9E9002300E76FF00100FDE66FF0AC
:103B90000800FAE6082CA1D9102CB4D9202CEED8B4
:103BA000C4E7BBF1000FAED0022384E7BBF1000FE6
:103BB000BCD004237FE70000012A30B5144638BF8B
:103BC000012485B00025402C28BF4024012ACDE9DE
:103BD000025518D81B788DF8083063070AD004AB5B
:103BE000624203EBD40502F0070215F8083C93404B
:103BF00005F8083C034600912246002102A8FFF781
:103C00005BFB05B030BD082AE4D9102A03D81B8815
:103C1000ADF80830E1E7202A95BF1B68D3E90023FF
:103C20000293CDE90223D8E710B5CB681BB98B60AE
:103C30000B618B8210BDC4681A681C60C360438A24
:103C4000013B4382CA60F0E72DE9F04FD1F80080D4
:103C500093B004460D4618F0800FCDE90323C8F356
:103C6000C01219BFC8F3C03BC8F306264FF0020BC1
:103C70001646B8F1000F80F2D18118F0C0430593C9
:103C800040F0CC810B7B002B00F0C881BBF1020F10
:103C900003D00178B14240F0C48108F07F01069161
:103CA0006AB3C8F3074A2B447606069A46EA0B46DF
:103CB00093F8039046EA82465FEAD91346EA0A0679
:103CC000079300F090800022002367680AA920462D
:103CD000CDE90A23069B524600935B46B84700286D
:103CE0007ED0A7699FB9314604F10C00FFF746FB6F
:103CF0000746E0B96FF0020013B0BDE8F08FC8F3DB
:103D00000F2A18F07F0F08BF0AF0030ACBE73B69C0
:103D10009E420DD03F68002FF9D1314604F10C00CE
:103D2000FFF72CFB07460028E4D0A3693B60A7619E
:103D300000264FF6FF70DDE90A23C6F1200E22FAB5
:103D400006F1A6F1200C083603FA0EFE099223FABA
:103D50000CFC089341EA0E0141EA0C01C9B2FFF7DD
:103D6000E3FA402EDDE90832E7D1B882FB7D09F0A5
:103D70001F06C8F30468C3F384039B1B98B2002B8F
:103D8000D7E90221BCBF00F120031BB252EA0100B7
:103D90000FD00398821A049860EB0101A748904263
:103DA0004FF000028A4104D3079A002A5BD0012B0E
:103DB00023DDFA7D4FEA89033946204602F00302EB
:103DC00003F07C031343FB75FFF730FB079BA3B99C
:103DD000FB7DC3F38402013262F38603FB7504E0CA
:103DE0006FF00B0088E7A76917B96FF00C0083E745
:103DF0003B699E42BAD03F68F6E719F0400F32D0D7
:103E0000039B142200210DA8BB60049BFB60FDF7FF
:103E100081FF039B0AA920460A93049BADF83EA0AC
:103E20000B932B1D8DF840B00C932B7B8DF84160CC
:103E3000013B8DF84280DBB2ADF83C30069B8DF83B
:103E4000433094F8243083F001038DF84430A368A4
:103E50009847FB7DC3F38403013303F01F039B02E8
:103E6000FB82002048E7FB7DC9F34012B2EBD31F71
:103E700040F0DA80C3F38403B34240F0D88007995E
:103E80004FEA99122B7B002934D0D20741D4032B5F
:103E900040F2D080039BAE1D394604F10C00BB609C
:103EA0003246049BFB602B7B033BDBB2FFF7D0FA6F
:103EB00000280DDA20463946FFF7B8FAFB7D0320CB
:103EC000C3F38403013303F01F039B02FB8213E758
:103ED000AB883B832A7B033AD2B2B88A3146FFF7DC
:103EE00033FAFB7DB882DA43C2F3C01262F3C71320
:103EF000FB75B6E76AB92E1D013B394604F10C008B
:103F0000DBB23246FFF7A4FA0028D3DB2A7B013A62
:103F1000E2E7F98A013BC1F30901DAB2052959D870
:103F2000281D002307F11A0C9A4208D910F801EB5A
:103F300001330CF801E00131DBB20629F4D1039919
:103F400093420A9138BF043304992CBF002355FAD9
:103F500083F30B9107F11A010C9179680E930D917F
:103F6000291DFB8AADF83EA0C3F309038DF840B0CC
:103F70008DF841601A44069B8DF842808DF84330DD
:103F800094F82430ADF83C2083F001038DF84430E0
:103F90000023B88A7B602A7B013AFFF7D5F93B8B77
:103FA000B882834203D1A3680AA9204698472046D5
:103FB0000AA9FFF739FEFB7DB88AC3F384030133F6
:103FC00003F01F039B02FB823B8B984214BF11201E
:103FD000002091E67B68002BB1D0062001E01C3068
:103FE0006346D3F800C0BCF1000FF8D1091A05F1FF
:103FF000040C081D00EB030905989DF8143001EB33
:10400000000EBEF11B0F9AD89A4298D91CF8013BBA
:1040100009F8013B059B01330593EDE76FF00900BB
:104020006AE66FF00A0067E66FF00D0064E66FF075
:104030000E0061E66FF00F005EE600BF80841E0098
:10404000EFF30983054968334A6B22F001024A63A2
:1040500083F30988002383F31188704700EF00E0A1
:10406000202080F3118862B60D4B0E4AD96821F4E6
:10407000E0610904090C0A430B49DA60D3F8FC201B
:1040800042F08072C3F8FC20084AC2F8B01F1168E1
:1040900041F0010111601022DA7783F822007047A5
:1040A00000ED00E00003FA0555CEACC5001000E0BD
:1040B000202310B583F311880E4B5B6813F4006363
:1040C00014D0F1EE103AEFF309844FF08073683C9E
:1040D000E361094BDB6B236684F3098800F0C2FFC0
:1040E00010B1064BA36110BD054BFBE783F31188AC
:1040F000F9E700BF00ED00E000EF00E00B0700086B
:104100000E070008026843681143016003B11847B5
:1041100070470000024A136843F0C0031360704701
:104120000078004013B50E4C204600F0A1FA04F1CF
:10413000140000234FF400720A49009400F062F961
:10414000094B4FF40072094904F13800009400F063
:10415000DBF9074A074BC4E9172302B010BD00BFC3
:10416000D45E0020405F002015410008406100201F
:104170000078004000E1F505037C30B5244C0029AF
:1041800018BF0C46012B11D1224B98420ED1224B65
:10419000D3F8E82042F08042C3F8E820D3F8102199
:1041A00042F08042C3F81021D3F810312268036E28
:1041B000C16D03EB52038466B3FBF2F3626815042E
:1041C00042BF23F0070503F0070343EA4503CB6032
:1041D000A36843F040034B60E36843F001038B6046
:1041E00042F4967343F001030B604FF0FF330B6210
:1041F000510505D512F0102205D0B2F1805F04D030
:1042000080F8643030BD7F23FAE73F23F8E700BF32
:1042100008740008D45E0020004402582DE9F047DD
:10422000C66D05463768F4692107346219D014F069
:10423000080118BF8021E20748BF41F02001A30711
:104240004FF0200348BF41F04001600748BF41F4F0
:10425000807183F31188281DFFF754FF002383F337
:104260001188E2050AD5202383F311884FF40071E9
:10427000281DFFF747FF002383F311884FF0200923
:104280004FF0000A14F0200838D13B0616D54FF045
:10429000200905F1380A200610D589F31188504607
:1042A00000F066F9002836DA0821281DFFF72AFFFA
:1042B00027F080033360002383F31188790614D537
:1042C000620612D5202383F31188D5E913239A427D
:1042D00008D12B6C33B127F040071021281DFFF7C0
:1042E00011FF3760002383F31188E30618D5AA6E07
:1042F0001369ABB15069BDE8F047184789F31188DD
:10430000736A284695F86410194000F0CBF98AF3D7
:104310001188F469B6E7B06288F31188F469BAE7E6
:10432000BDE8F087090100F16043012203F5614314
:10433000C9B283F8001300F01F039A4043099B00A1
:1043400003F1604303F56143C3F880211A607047AD
:10435000F8B51546826804460B46AA4200D2856825
:10436000A1692669761AB5420BD218462A46FDF78E
:10437000ABFCA3692B44A3612846A3685B1BA36025
:10438000F8BD0CD9AF1B18463246FDF79DFC3A46E6
:10439000E1683044FDF798FCE3683B44EBE71846DE
:1043A0002A46FDF791FCE368E5E700008368934245
:1043B000F7B50446154600D28568D4E90460361A7C
:1043C000B5420BD22A46FDF77FFC63692B4463613B
:1043D0002846A3685B1BA36003B0F0BD0DD932462D
:1043E000AF1B0191FDF770FC01993A46E06831443A
:1043F000FDF76AFCE3683B44E9E72A46FDF764FC05
:10440000E368E4E710B50A440024C361029B8460BA
:10441000C16002610362C0E90000C0E9051110BD7E
:1044200008B5D0E90532934201D1826882B9826829
:10443000013282605A1C426119700021D0E90432B5
:104440009A4224BFC368436100F0E6FE002008BD25
:104450004FF0FF30FBE7000070B5202304460E4606
:1044600083F31188A568A5B1A368A269013BA36085
:10447000531CA36115782269934224BFE368A361AA
:10448000E3690BB120469847002383F3118828463F
:1044900007E03146204600F0AFFE0028E2DA85F35F
:1044A000118870BD2DE9F74F04460E461746984611
:1044B000D0F81C904FF0200A8AF311884FF0000BBF
:1044C000154665B12A4631462046FFF741FF0346AF
:1044D00060B94146204600F08FFE0028F1D000234D
:1044E00083F31188781B03B0BDE8F08FB9F1000F9A
:1044F00003D001902046C847019B8BF31188ED1A29
:104500001E448AF31188DCE7C160C361009B8260AE
:104510000362C0E905111144C0E900000161704760
:10452000F8B504460D461646202383F31188A76884
:10453000A7B1A368013BA36063695A1C62611D7047
:10454000D4E904329A4224BFE3686361E3690BB1A2
:1045500020469847002080F3118807E03146204626
:1045600000F04AFE0028E2DA87F31188F8BD000067
:10457000D0E9052310B59A4201D182687AB98268E0
:104580000021013282605A1C82611C7803699A42C0
:1045900024BFC368836100F03FFE204610BD4FF08A
:1045A000FF30FBE72DE9F74F04460E4617469846C5
:1045B000D0F81C904FF0200A8AF311884FF0000BBE
:1045C000154665B12A4631462046FFF7EFFE034601
:1045D00060B94146204600F00FFE0028F1D00023CC
:1045E00083F31188781B03B0BDE8F08FB9F1000F99
:1045F00003D001902046C847019B8BF31188ED1A28
:104600001E448AF31188DCE70268436811430160A5
:1046100003B11847704700001430FFF743BF000094
:104620004FF0FF331430FFF73DBF00003830FFF785
:10463000B9BF00004FF0FF333830FFF7B3BF0000C1
:104640001430FFF709BF00004FF0FF311430FFF7BF
:1046500003BF00003830FFF763BF00004FF0FF32A8
:104660003830FFF75DBF000000207047FFF75ABDEC
:10467000044B036000234360C0E902330123037449
:10468000704700BF2074000810B52023044683F350
:104690001188FFF771FD02232374002383F311882F
:1046A00010BD000038B5C36904460D461BB904218E
:1046B0000844FFF7A9FF294604F11400FFF7B0FEF4
:1046C000002806DA201D4FF48061BDE83840FFF76E
:1046D0009BBF38BD026843681143016003B11847AE
:1046E0007047000013B5406B00F58054D4F8A4382F
:1046F0001A681178042914D1017C022911D1197981
:10470000012312898B4013420BD101A94C3002F0D6
:104710009BF8D4F8A4480246019B2179206800F058
:10472000DFF902B010BD0000143002F01DB8000027
:104730004FF0FF33143002F017B800004C3002F095
:10474000EFB800004FF0FF334C3002F0E9B8000042
:10475000143001F0EBBF00004FF0FF31143001F0D6
:10476000E5BF00004C3002F0BBB800004FF0FF3254
:104770004C3002F0B5B800000020704710B500F5CD
:104780008054D4F8A4381A681178042917D1017C10
:10479000022914D15979012352898B4013420ED139
:1047A000143001F07DFF024648B1D4F8A4484FF41C
:1047B000407361792068BDE8104000F07FB910BDFA
:1047C000406BFFF7DBBF0000704700007FB5124B66
:1047D00001250426044603600023057400F18402C9
:1047E00043602946C0E902330C4B02901430019318
:1047F0004FF44073009601F02FFF094B04F69442EA
:10480000294604F14C000294CDE900634FF4407353
:1048100001F0F6FF04B070BD48740008C1470008FD
:10482000E54600080A68202383F311880B790B33CF
:1048300042F823004B79133342F823008B7913B1EC
:104840000B3342F8230000F58053C3F8A418022369
:104850000374002383F311887047000038B5037F89
:10486000044613B190F85430ABB90125201D022144
:10487000FFF730FF04F114006FF00101257700F01D
:10488000D7FC04F14C0084F854506FF00101BDE8EE
:10489000384000F0CDBC38BD10B5012104460430CD
:1048A000FFF718FF0023237784F8543010BD000071
:1048B00038B504460025143001F0E6FE04F14C0042
:1048C000257701F0B5FF201D84F854500121FFF732
:1048D00001FF2046BDE83840FFF750BF90F8803018
:1048E00003F06003202B06D190F881200023212AB9
:1048F00003D81F2A06D800207047222AFBD1C0E91E
:104900001D3303E0034A426707228267C367012021
:10491000704700BF3422002037B500F58055D5F828
:10492000A4381A68117804291AD1017C022917D1F8
:104930001979012312898B40134211D100F14C04E3
:10494000204602F035F858B101A9204601F07CFF5D
:10495000D5F8A4480246019B2179206800F0C0F8F0
:1049600003B030BD01F10B03F0B550F8236085B002
:1049700004460D46FEB1202383F3118804EB85071E
:10498000301D0821FFF7A6FEFB6806F14C005B69AD
:104990001B681BB1019001F065FF019803A901F0AC
:1049A00053FF024648B1039B2946204600F098F881
:1049B000002383F3118805B0F0BDFB685A691268C3
:1049C000002AF5D01B8A013B1340F1D104F180028B
:1049D000EAE70000133138B550F82140ECB120234C
:1049E00083F3118804F58053D3F8A428136852790F
:1049F00003EB8203DB689B695D6845B104216018A5
:104A0000FFF768FE294604F1140001F053FE20462A
:104A1000FFF7B4FE002383F3118838BD7047000010
:104A200001F05CB901234022002110B5044600F8D2
:104A3000303BFDF76FF90023C4E9013310BD0000DE
:104A400010B52023044683F31188242241600021FD
:104A50000C30FDF75FF9204601F062F90223237064
:104A6000002383F3118810BD70B500EB8103054668
:104A700050690E461446DA6018B110220021FDF785
:104A800049F9A06918B110220021FDF743F9314618
:104A90002846BDE8704001F055BA00008368202226
:104AA000002103F0011310B5044683601030FDF7B8
:104AB00031F92046BDE8104001F0D0BAF0B401252C
:104AC00000EB810447898D40E4683D43A46945813A
:104AD00023600023A2606360F0BC01F0EDBA000027
:104AE000F0B4012500EB810407898D40E4683D4363
:104AF0006469058123600023A2606360F0BC01F05B
:104B000063BB000070B50223002504462422037015
:104B10002946C0F888500C3040F8045CFDF7FAF8DC
:104B2000204684F8705001F0A1F963681B6823B136
:104B300029462046BDE87040184770BD037880F8CC
:104B40008C300523037043681B6810B504460BB115
:104B5000042198470023A36010BD000090F88C202A
:104B6000436802701B680BB10521184770470000AD
:104B700070B590F87030044613B1002380F870309F
:104B800004F18002204601F08DFA63689B68B3B996
:104B900094F8803013F0600535D00021204601F0F4
:104BA00037FD0021204601F027FD63681B6813B123
:104BB000062120469847062384F8703070BD2046B1
:104BC00098470028E4D0B4F88630A26F9A4288BF94
:104BD000A36794F98030A56F002B4FF0200380F27B
:104BE0000381002D00F0F280092284F8702083F305
:104BF000118800212046D4E91D23FFF771FF00230F
:104C000083F31188DAE794F8812003F07F0343EA05
:104C1000022340F20232934200F0C58021D8B3F55E
:104C2000807F48D00DD8012B3FD0022B00F093801D
:104C3000002BB2D104F1880262670222A267E36707
:104C4000C1E7B3F5817F00F09B80B3F5407FA4D12D
:104C500094F88230012BA0D1B4F8883043F00203DD
:104C600032E0B3F5006F4DD017D8B3F5A06F31D057
:104C7000A3F5C063012B90D86368204694F8822086
:104C80005E6894F88310B4F88430B047002884D06C
:104C9000436863670368A3671AE0B3F5106F36D003
:104CA00040F6024293427FF478AF5C4B6367022385
:104CB000A3670023C3E794F88230012B7FF46DAF24
:104CC000B4F8883023F00203A4F88830C4E91D55F5
:104CD000E56778E7B4F88030B3F5A06F0ED194F8AB
:104CE0008230204684F88A3001F01EF963681B6820
:104CF00013B1012120469847032323700023C4E900
:104D00001D339CE704F18B0363670123C3E723781A
:104D1000042B10D1202383F311882046FFF7BEFE19
:104D200085F311880321636884F88B5021701B6818
:104D30000BB12046984794F88230002BDED084F8DF
:104D40008B300423237063681B68002BD6D00221AC
:104D500020469847D2E794F8843020461D0603F099
:104D60000F010AD501F090F9012804D002287FF440
:104D700014AF2B4B9AE72B4B98E701F077F9F3E749
:104D800094F88230002B7FF408AF94F8843013F04D
:104D90000F01B3D01A06204602D501F051FCADE751
:104DA00001F042FCAAE794F88230002B7FF4F5AEC4
:104DB00094F8843013F00F01A0D01B06204602D5D2
:104DC00001F026FC9AE701F017FC97E7142284F81B
:104DD000702083F311882B462A4629462046FFF788
:104DE0006DFE85F31188E9E65DB1152284F8702027
:104DF00083F3118800212046D4E91D23FFF75EFECE
:104E0000FDE60B2284F8702083F311882B462A4696
:104E100029462046FFF764FEE3E700BF78740008E8
:104E2000707400087474000838B590F87030044647
:104E3000002B3ED0063BDAB20F2A34D80F2B32D8E3
:104E4000DFE803F03731310822323131313131318D
:104E500031313737856FB0F886309D4214D2C36840
:104E60001B8AB5FBF3F203FB12556DB9202383F3C4
:104E700011882B462A462946FFF732FE85F3118812
:104E80000A2384F870300EE0142384F87030202355
:104E900083F31188002320461A461946FFF70EFEB9
:104EA000002383F3118838BDC36F03B198470023F3
:104EB000E7E70021204601F0ABFB0021204601F08E
:104EC0009BFB63681B6813B10621204698470623A5
:104ED000D7E7000010B590F870300446142B29D0A5
:104EE00017D8062B05D001D81BB110BD093B022BEA
:104EF000FBD80021204601F08BFB0021204601F069
:104F00007BFB63681B6813B1062120469847062384
:104F100019E0152BE9D10B2380F87030202383F39F
:104F2000118800231A461946FFF7DAFD002383F3A0
:104F30001188DAE7C3689B695B68002BD5D1C36F22
:104F400003B19847002384F87030CEE7024B00226B
:104F5000C3E900339A6070474063002000238268F1
:104F60000374054B1B6899689142FBD25A68036031
:104F700042601060586070474063002008B52023ED
:104F800083F31188037C032B05D0042B0DD02BB9A0
:104F900083F3118808BD436900221A604FF0FF3384
:104FA0004361FFF7DBFF0023F2E7D0E90032136033
:104FB0005A60F3E7002382680374054B1B68996805
:104FC0009142FBD85A680360426010605860704795
:104FD00040630020054B1969087418680268536023
:104FE0001A60186101230374FBF77ABB4063002049
:104FF0004B1C30B5044687B00A4D10D02B6901A870
:10500000094A00F031F92046FFF7E4FF049B13B191
:1050100001A800F065F92B69586907B030BDFFF7AA
:10502000D9FFF8E7406300207D4F000838B50C4DEC
:10503000044641612B6981689A68914203D8BDE8B2
:105040003840FFF78BBF1846FFF7B4FF01232C61F0
:10505000014623742046BDE83840FBF741BB00BF42
:1050600040630020044B1A681B6990689B68984253
:1050700094BF0020012070474063002010B5084C09
:10508000236820691A6854602260012223611A741F
:10509000FFF790FF01462069BDE81040FBF720BBF9
:1050A0004063002008B5FFF7DDFF18B1BDE80840F8
:1050B000FFF7E4BF08BD0000FFF7E0BFFEE7000018
:1050C00010B50C4CFFF742FF00F0C0F880220A49EF
:1050D000204600F047F8012344F8180C0374FEF74B
:1050E000BFFF002383F3118862B60448BDE8104077
:1050F00000F058B8686300207C7400088C740008C5
:1051000008B572B6034B586200F008FC00F0D6FCFC
:10511000FEE700BF4063002000F01CB9EFF31180F0
:1051200020B9EFF30583202282F311887047000035
:1051300010B530B9EFF30584C4F3080414B180F35B
:10514000118810BDFFF7AEFF84F31188F9E7000066
:10515000034A516853685B1A9842FBD8704700BFF6
:10516000001000E082600222028270478368A3F18F
:105170007C0243F80C2C026943F83C2C426943F84A
:10518000382C074A43F81C2CC268A3F1180043F8D6
:10519000102C022203F8082C002203F8072C704779
:1051A000F906000810B5202383F31188FFF7DEFF0E
:1051B00000210446FFF73AFF002383F311882046BD
:1051C00010BD0000024B1B6958610F20FFF702BFA2
:1051D00040630020202383F31188FFF7F3BF000012
:1051E00008B50146202383F311880820FFF700FF4C
:1051F000002383F3118808BD49B1064B42681B693F
:1052000018605A60136043600420FFF7F1BE4FF04E
:10521000FF307047406300200368984206D01A6848
:105220000260506018465961FFF798BE7047000051
:1052300038B504460D462068844200D138BD036865
:1052400023605C604561FFF789FEF4E7054B4FF092
:10525000FF3103F11402C3E905220022C3E907125A
:10526000704700BF4063002070B51C4E05460C46D9
:10527000C0E9032301F0D2FB334653F8142F9A42BE
:105280000DD130620A2C2CBF00190A302A60C5E902
:105290000124C6E90555BDE8704001F0A9BB316A9B
:1052A000431AE31838BF1C469368A34202D9081971
:1052B00001F0AEFB73699A6894420CD85A68AC60EE
:1052C0002B606A6015609A685D60121B9A604FF0EF
:1052D000FF33F36170BDA41A1B68ECE74063002044
:1052E00038B51B4C636998420DD08168D0E9003213
:1052F00013605A600022C2609A680A449A604FF0B4
:10530000FF33E36138BD03682246002142F8143FB1
:1053100093425A60C16003D1BDE8384001F072BBCE
:105320009A688168256A0A449A6001F077FB63698C
:10533000411B9A688A42E5D9AB181D1A206A092DCB
:1053400098BF01F10A02BDE83840104401F060BB8B
:10535000406300202DE9F041184C002704F11406A9
:10536000656901F05BFB236AAA68C11A8A4215D8F5
:105370001344D5F80C802362D5E9003213605A60DB
:105380006369EF60B34201D101F03CFB87F3118800
:105390002869C047202383F31188E1E76169B1429E
:1053A00009D013441B1ABDE8F0410A2B2CBFC018CA
:1053B0000A3001F02DBBBDE8F08100BF4063002042
:1053C00000207047FEE70000704700004FF0FF30FC
:1053D0007047000002290CD0032904D00129074896
:1053E00018BF00207047032A05D8054800EBC2000B
:1053F0007047044870470020704700BF7075000870
:10540000442200202475000870B59AB0054608466D
:10541000144601A900F0C2F801A8FCF773FC431C74
:105420000022C6B25B001046C5E900342370032396
:10543000023404F8013C01ABD1B202348E4201D8EF
:105440001AB070BD13F8011B013204F8010C04F806
:10545000021CF1E708B5202383F311880348FFF706
:105460005BFA002383F3118808BD00BFF8640020B5
:1054700090F8803003F01F02012A07D190F88120B4
:105480000B2A03D10023C0E91D3315E003F06003AC
:10549000202B08D1B0F884302BB990F88120212A34
:1054A00003D81F2A04D8FFF719BA222AEBD0FAE74B
:1054B000034A426707228267C3670120704700BF23
:1054C0003B22002007B5052917D8DFE801F019169F
:1054D00003191920202383F31188104A0121019018
:1054E000FFF7C2FA019802210D4AFFF7BDFA0D48F5
:1054F000FFF7DEF9002383F3118803B05DF804FBA6
:10550000202383F311880748FFF7A8F9F2E7202347
:1055100083F311880348FFF7BFF9EBE7C474000871
:10552000E8740008F864002038B50C4D0C4C2A468D
:105530000C4904F10800FFF767FF05F1CA0204F106
:1055400010000949FFF760FF05F5CA7204F1180061
:105550000649BDE83840FFF757BF00BFD07D0020A7
:1055600044220020A4740008AE740008B974000836
:1055700070B5044608460D46FCF7C4FBC6B220468B
:10558000013403780BB9184670BD32462946FCF742
:10559000A5FB0028F3D10120F6E700002DE9F04734
:1055A00005460C46FCF7AEFB2B49C6B22846FFF772
:1055B000DFFF08B10A36F6B228492846FFF7D8FFC0
:1055C00008B11036F6B2632E0BD8DFF88C80DFF806
:1055D0008C90234FDFF894A02E7846B92670BDE852
:1055E000F08729462046BDE8F04701F03BBE252E56
:1055F0002ED1072241462846FCF770FB70B9194BA3
:10560000224603F1100153F8040B8B4242F8040BBD
:10561000F9D11B78073511341370DDE708224946AC
:105620002846FCF75BFB98B9A21C0F4B1978023295
:105630000909C95D02F8041C13F8011B01F00F01F0
:105640005345C95D02F8031CF0D118340835C3E78F
:10565000013504F8016BBFE790750008B9740008C4
:1056600098750008A272000800E8F11F0CE8F11F0D
:10567000BFF34F8F044B1A695107FCD1D3F81021A7
:105680005207F8D1704700BF0020005208B50D4BFB
:105690001B78ABB9FFF7ECFF0B4BDA68D10704D5E9
:1056A0000A4A5A6002F188325A60D3F80C21D207B4
:1056B00006D5064AC3F8042102F18832C3F8042152
:1056C00008BD00BF2E800020002000522301674546
:1056D00008B5114B1B78F3B9104B1A69510703D564
:1056E000DA6842F04002DA60D3F81021520705D59B
:1056F000D3F80C2142F04002C3F80C21FFF7B8FFA9
:10570000064BDA6842F00102DA60D3F80C2142F06D
:105710000102C3F80C2108BD2E8000200020005299
:105720000F289ABF00F580604004002070470000F9
:105730004FF4003070470000102070470F2808B564
:105740000BD8FFF7EDFF00F500330268013204D1FA
:1057500004308342F9D1012008BD0020FCE700009D
:105760000F2870B5054645D8FFF7D8FC224CFFF747
:105770007FFF0646FFF78AFF4FF0FF33072D636177
:10578000C4F8143120D82361FFF772FF2B0243F0D5
:105790002403E360E36843F08003E36023695A076E
:1057A000FCD42846FFF764FF4FF40031FFF7B8FF41
:1057B00000F060F93046FFF78BFFFFF7B9FC284691
:1057C000BDE87040FFF7BABFC4F81031FFF750FFD3
:1057D000A5F108031B0243F02403C4F80C31D4F8EC
:1057E0000C3143F08003C4F80C31D4F810315B075E
:1057F000FBD4D6E7002070BD002000522DE9F84F01
:1058000040EA020305460C461746D80602D000209F
:10581000BDE8F88F27F01F07DFF8D4B0FFF736FF99
:105820002744BC4203D10120FFF752FFF0E72022BA
:105830002946204601F098FC10B920352034F0E7C5
:105840002B4605F120021E68711CE0D104339A42F8
:10585000F9D1FFF763FC05F17843234AB3F5801FC4
:10586000224B28BF9A4603F1040338BF9046A2F1A9
:10587000080228BF9846A3F108033ABF9146DA46CA
:105880009946FFF7F5FEC8F80060A5EB040CD9F8BF
:10589000002004F11C0142F00202C9F80020221F7E
:1058A000DAF8006016F00506FAD152F8043F8A4291
:1058B0004CF80230F4D1BFF34F8FFFF7D9FE4FF011
:1058C000FF32C8F80020D9F8002022F00202C9F8FF
:1058D0000020FFF72DFC20222146284601F044FC41
:1058E0000028AAD030469FE7142000521021005211
:1058F0001020005210B5084C237828B11BB9FFF7CF
:10590000C5FE0123237010BD002BFCD02070BDE824
:105910001040FFF7DDBE00BF2E80002038B5054DDA
:1059200000240334696855F80C0B00F0B5F8122C0C
:10593000F7D138BDAC75000870B5104E82B0FFF7D6
:10594000EDFB054601F06AF8326803469042336089
:1059500037BF0B4A0A495168146836BF0131D1E993
:10596000004151600419284641F100010191FFF7FF
:10597000DFFB2046019902B070BD00BF30800020DF
:105980003880002070B5124E82B0FFF7C7FB054685
:1059900001F044F8326803469042336037BF0D4A45
:1059A0000C495168146836BF0131D1E9004151609A
:1059B0000419284641F100010191FFF7B9FB4FF4AA
:1059C0007A72002320460199FAF772FC02B070BD8A
:1059D00030800020388000200244074BD2B210B53E
:1059E000904200D110BD441C00B253F8200041F891
:1059F000040BE0B2F4E700BF504000580E4B30B546
:105A00001C6F240405D41C6F1C671C6F44F40044F5
:105A10001C670A4C02442368D2B243F480732360AB
:105A2000074B904200D130BD441C51F8045B00B2DA
:105A300043F82050E0B2F4E700440258004802580E
:105A40005040005807B5012201A90020FFF7C4FF0C
:105A5000019803B05DF804FB13B50446FFF7F2FFAD
:105A6000A04205D0012201A900200194FFF7C6FF42
:105A700002B010BD0144BFF34F8F064B884204D3E0
:105A8000BFF34F8FBFF36F8F7047C3F85C022030B6
:105A9000F4E700BF00ED00E00144BFF34F8F064B79
:105AA000884204D3BFF34F8FBFF36F8F7047C3F8A3
:105AB00070022030F4E700BF00ED00E07047000006
:105AC000074B45F255521A6002225A6040F6FF72A7
:105AD0009A604CF6CC421A600122024B1A70704751
:105AE0000048005844800020034B1B781BB1034B37
:105AF0004AF6AA221A6070474480002000480058E5
:105B0000034B1A681AB9034AD2F8D0241A607047B6
:105B10004080002000400258024B4FF48032C3F80E
:105B2000D02470470040025808B5FFF7E9FF024B48
:105B30001868C0F3806008BD4080002070B5BFF3D6
:105B40004F8FBFF36F8F1A4A0021C2F85012BFF374
:105B50004F8FBFF36F8F536943F400335361BFF32B
:105B60004F8FBFF36F8FC2F88410BFF34F8FD2F8FF
:105B7000803043F6E074C3F3C900C3F34E335B01D6
:105B800003EA0406014646EA81750139C2F860520B
:105B9000F9D2203B13F1200FF2D1BFF34F8F53699D
:105BA00043F480335361BFF34F8FBFF36F8F70BDEA
:105BB00000ED00E0FEE700000A4B0B480B4A904264
:105BC0000BD30B4BC11EDA1C121A22F003028B42BC
:105BD00038BF00220021FCF79DB853F8041B40F8A1
:105BE000041BECE738780008208200202082002087
:105BF000208200207047000070B5D0E924430022C5
:105C00004FF0FF359E6804EB42135101D3F80009B1
:105C1000002805DAD3F8000940F08040C3F80009F5
:105C2000D3F8000B002805DAD3F8000B40F08040D1
:105C3000C3F8000B013263189642C3F80859C3F841
:105C4000085BE0D24FF00113C4F81C3870BD0000AF
:105C500000EB8103D3F80CC02DE9F043DCF81420ED
:105C60004E1CD0F89050D2F800E005EB063605EB5C
:105C70004118506870450AD30122D5F8343802FA29
:105C800001F123EA0101C5F83418BDE8F083AEEB59
:105C90000003BCF81040A34228BF2346D8F8184997
:105CA000A4B2B3EB840FF0D89468A4F1040959F8B6
:105CB000047F3760A4EB09071F44042FF7D81C4466
:105CC000034494605360D4E7890141F020010161ED
:105CD00003699B06FCD41220FFF73ABA10B50A4CB0
:105CE0002046FEF79FFE094BC4F89030084BC4F8DD
:105CF0009430084C2046FEF795FE074BC4F89030D0
:105D0000064BC4F8943010BD4880002000000840C5
:105D100018760008E4800020000004402476000883
:105D200070B503780546012B5DD1494BD0F8904002
:105D3000984259D1474B0E216520D3F8D82042F024
:105D40000062C3F8D820D3F8002142F00062C3F803
:105D50000021D3F80021D3F8802042F00062C3F87C
:105D60008020D3F8802022F00062C3F88020D3F88E
:105D70008030FEF7D7FA384BE360384BC4F8003870
:105D80000023D5F89060C4F8003EC02323604FF490
:105D90000413A3633369002BFCDA01230C20336165
:105DA000FFF7D6F93369DB07FCD41220FFF7D0F9EF
:105DB0003369002BFCDA00262846A660FFF71CFF9B
:105DC0006B68C4F81068DB68C4F81468C4F81C6811
:105DD000002B3AD1224BA3614FF0FF336361A368DC
:105DE00043F00103A36070BD1E4B9842C8D1194B0C
:105DF0000E214D20D3F8D82042F00072C3F8D820ED
:105E0000D3F8002142F00072C3F80021D3F800213A
:105E1000D3F8802042F00072C3F88020D3F88020AD
:105E200022F00072C3F88020D3F88020D3F8D82065
:105E300022F08062C3F8D820D3F8002122F08062DB
:105E4000C3F80021D3F8003193E7074BC3E700BF45
:105E50004880002000440258401400400300200203
:105E6000003C30C0E4800020083C30C0F8B5D0F8D9
:105E70009040054600214FF000662046FFF724FFC2
:105E8000D5F8941000234FF001128F684FF0FF30C7
:105E9000C4F83438C4F81C2804EB431201339F4281
:105EA000C2F80069C2F8006BC2F80809C2F8080B12
:105EB000F2D20B68D5F89020C5F8983063621023B1
:105EC0001361166916F01006FBD11220FFF740F996
:105ED000D4F8003823F4FE63C4F80038A36943F40F
:105EE000402343F01003A3610923C4F81038C4F819
:105EF00014380B4BEB604FF0C043C4F8103B094B18
:105F0000C4F8003BC4F81069C4F80039D5F89830DB
:105F100003F1100243F48013C5F89820A362F8BD82
:105F2000F475000840800010D0F8902090F88A1096
:105F3000D2F8003823F4FE6343EA0113C2F80038B4
:105F4000704700002DE9F84300EB8103D0F8905032
:105F50000C468046DA680FFA81F94801166806F0A7
:105F60000306731E022B05EB41134FF0000194BF93
:105F7000B604384EC3F8101B4FF0010104F11003B2
:105F800098BF06F1805601FA03F3916998BF06F5B0
:105F9000004600293AD0578A04F158013743490195
:105FA0006F50D5F81C180B430021C5F81C382B186E
:105FB0000127C3F81019A7405369611E9BB3138AC8
:105FC000928B9B08012A88BF5343D8F898209818D1
:105FD00042EA034301F140022146C8F898002846EE
:105FE00005EB82025360FFF76FFE08EB8900C36880
:105FF0001B8A43EA845348341E4364012E51D5F86A
:106000001C381F43C5F81C78BDE8F88305EB491719
:10601000D7F8001B21F40041C7F8001BD5F81C1865
:1060200021EA0303C0E704F13F030B4A2846214657
:1060300005EB83035A60FFF747FE05EB4910D0F8E4
:10604000003923F40043C0F80039D5F81C3823EA9E
:106050000707D7E70080001000040002D0F8942062
:106060001268C0F89820FFF7C7BD00005831D0F87B
:10607000903049015B5813F4004004D013F4001F22
:106080000CBF0220012070474831D0F89030490100
:106090005B5813F4004004D013F4001F0CBF02201F
:1060A0000120704700EB8101CB68196A0B6813600F
:1060B0004B6853607047000000EB810330B5DD682A
:1060C000AA691368D36019B9402B84BF40231360B9
:1060D0006B8A1468D0F890201C4402EB4110013CFC
:1060E00009B2B4FBF3F46343033323F0030343EA3D
:1060F000C44343F0C043C0F8103B2B6803F00303D4
:10610000012B0ED1D2F8083802EB411013F4807F36
:10611000D0F8003B14BF43F0805343F00053C0F865
:10612000003B02EB4112D2F8003B43F00443C2F8BB
:10613000003B30BD2DE9F041D0F8906005460C469B
:1061400006EB4113D3F8087B3A07C3F8087B08D560
:10615000D6F814381B0704D500EB8103DB685B68B5
:106160009847FA071FD5D6F81438DB071BD505EB7F
:106170008403D968CCB98B69488A5A68B2FBF0F6B7
:1061800000FB16228AB91868DA6890420DD2121AFA
:10619000C3E90024202383F3118821462846FFF712
:1061A0008BFF84F31188BDE8F081012303FA04F228
:1061B0006B8923EA02036B81CB68002BF3D0214665
:1061C0002846BDE8F041184700EB81034A0170B54D
:1061D000DD68D0F890306C692668E66056BB1A44DA
:1061E0004FF40020C2F810092A6802F00302012AC5
:1061F0000AB20ED1D3F8080803EB421410F4807FE2
:10620000D4F8000914BF40F0805040F00050C4F8AA
:10621000000903EB4212D2F8000940F00440C2F832
:1062200000090122D3F8340802FA01F10143C3F84E
:10623000341870BD19B9402E84BF402020602068FA
:106240001A442E8A8419013CB4FBF6F440EAC44097
:1062500040F00050C6E700002DE9F041D0F8906012
:1062600004460D4606EB4113D3F80879C3F80879C4
:10627000FB071CD5D6F81038DA0718D500EB8103D8
:10628000D3F80CC0DCF81430D3F800E0DA68964597
:106290001BD2A2EB0E024FF000081A60C3F8048074
:1062A000202383F31188FFF78FFF88F311883B06C3
:1062B00018D50123D6F83428AB40134212D0294612
:1062C0002046BDE8F041FFF7C3BC012303FA01F209
:1062D000038923EA02030381DCF80830002BE6D0AF
:1062E0009847E4E7BDE8F0812DE9F84FD0F89050E9
:1062F00004466E69AB691E4016F480586E6103D087
:10630000BDE8F84FFEF7FEBB002E12DAD5F8003ECE
:106310009F0705D0D5F8003E23F00303C5F8003EE3
:10632000D5F80438204623F00103C5F80438FEF7F9
:1063300015FC300505D52046FFF75EFC2046FEF72C
:10634000FDFBB1040CD5D5F8083813F0060FEB6847
:1063500023F470530CBF43F4105343F4A053EB6089
:10636000320704D56368DB680BB120469847F30217
:1063700000F1BA80B70226D5D4F8909000274FF0EC
:10638000010A09EB4712D2F8003B03F44023B3F5AE
:10639000802F11D1D2F8003B002B0DDA62890AFA66
:1063A00007F322EA0303638104EB8703DB68DB68FE
:1063B00013B13946204698470137D4F89430FFB2DC
:1063C0009B689F42DDD9F00619D5D4F89000026A87
:1063D000C2F30A1702F00F0302F4F012B2F5802F95
:1063E00000F0CC80B2F5402F09D104EB83030022EA
:1063F00000F58050DB681B6A974240F0B2803003A2
:10640000D5F8185835D5E90303D500212046FFF704
:1064100091FEAA0303D501212046FFF78BFE6B03F3
:1064200003D502212046FFF785FE2F0303D5032164
:106430002046FFF77FFEE80203D504212046FFF740
:1064400079FEA90203D505212046FFF773FE6A02F3
:1064500003D506212046FFF76DFE2B0203D5072149
:106460002046FFF767FEEF0103D508212046FFF71E
:1064700061FE700340F1A980E90703D500212046A1
:10648000FFF7EAFEAA0703D501212046FFF7E4FE45
:106490006B0703D502212046FFF7DEFE2F0703D549
:1064A00003212046FFF7D8FEEE0603D5042120463F
:1064B000FFF7D2FEA80603D505212046FFF7CCFE44
:1064C000690603D506212046FFF7C6FE2A0603D536
:1064D00007212046FFF7C0FEEB0576D520460821B0
:1064E000BDE8F84FFFF7B8BED4F8909000274FF002
:1064F000010AD4F894305FFA87FB9B689B453FF60E
:1065000039AF09EB4B13D3F8002902F44022B2F55E
:10651000802F24D1D3F80029002A20DAD3F80029CB
:1065200042F09042C3F80029D3F80029002AFBDB8F
:106530005946D4F89000FFF7C7FB22890AFA0BF3FB
:1065400022EA0303238104EB8B03DB689B6813B10E
:1065500059462046984759462046FFF779FB0137B0
:10656000C7E7910701D1D0F80080072A02F10102A4
:106570009CBF03F8018B4FEA18283DE704EB830327
:1065800000F58050DA68D2F818C0DCF80820DCE9A1
:10659000001CA1EB0C0C00218F4208D1DB689B6929
:1065A0009A683A449A605A683A445A6027E711F068
:1065B000030F01D1D0F800808C4501F1010184BFA7
:1065C00002F8018B4FEA1828E6E7BDE8F88F0000D3
:1065D00008B50348FFF788FEBDE80840FDF768BD31
:1065E0004880002008B50348FFF77EFEBDE808405C
:1065F000FDF75EBDE4800020D0F8903003EB411140
:10660000D1F8003B43F40013C1F8003B7047000091
:10661000D0F8903003EB4111D1F8003943F4001366
:10662000C1F8003970470000D0F8903003EB4111F9
:10663000D1F8003B23F40013C1F8003B7047000081
:10664000D0F8903003EB4111D1F8003923F4001356
:10665000C1F800397047000030B50433039C017263
:10666000002104FB0325C160C0E90653049B0363BA
:10667000059BC0E90000C0E90422C0E90842C0E966
:106680000A11436330BD00000022416AC260C0E9C4
:106690000411C0E90A226FF00101FEF7C9BD000034
:1066A000D0E90432934201D1C2680AB9181D70477B
:1066B00000207047036919600021C2680132C2607E
:1066C000C269134482699342036124BF436A036130
:1066D000FEF7A2BD38B504460D46E3683BB16269DA
:1066E0000020131D1268A3621344E36207E0237ABB
:1066F00033B929462046FEF77FFD0028EDDA38BD84
:106700006FF00100FBE70000C368C269013BC36092
:106710004369134482699342436124BF436A4361DE
:1067200000238362036B03B11847704770B52023C1
:10673000044683F31188866A3EB9FFF7CBFF05460E
:1067400018B186F31188284670BDA36AE26A13F86F
:10675000015B9342A36202D32046FFF7D5FF0023DB
:1067600083F31188EFE700002DE9F84F04460E4649
:10677000174698464FF0200989F311880025AA464C
:10678000D4F828B0BBF1000F09D141462046FFF7ED
:10679000A1FF20B18BF311882846BDE8F88FD4E91A
:1067A0000A12A7EB050B521A934528BF9346BBF17B
:1067B000400F1BD9334601F1400251F8040B9142BE
:1067C00043F8040BF9D1A36A403640354033A36245
:1067D000D4E90A239A4202D32046FFF795FF8AF3B1
:1067E0001188BD42D8D289F31188C9E730465A468C
:1067F000FBF76AFAA36A5E445D445B44A362E7E781
:1068000010B5029C0433017204FB0321C460C0E98B
:1068100006130023C0E90A33039B0363049BC0E90A
:106820000000C0E90422C0E90842436310BD000033
:10683000026A6FF00101C260426AC0E904220022CC
:10684000C0E90A22FEF7F4BCD0E904239A4201D140
:10685000C26822B9184650F8043B0B60704700200C
:1068600070470000C3680021C2690133C3604369F7
:10687000134482699342436124BF436A4361FEF734
:10688000CBBC000038B504460D46E3683BB1236934
:1068900000201A1DA262E2691344E36207E0237A32
:1068A00033B929462046FEF7A7FC0028EDDA38BDAB
:1068B0006FF00100FBE7000003691960C268013A4C
:1068C000C260C269134482699342036124BF436A70
:1068D000036100238362036B03B118477047000014
:1068E00070B520230D460446114683F31188866A4D
:1068F0002EB9FFF7C7FF10B186F3118870BDA36AE8
:106900001D70A36AE26A01339342A36204D3E16972
:1069100020460439FFF7D0FF002080F31188EDE70F
:106920002DE9F84F04460D46904699464FF0200A4F
:106930008AF311880026B346A76A4FB94946204614
:10694000FFF7A0FF20B187F311883046BDE8F88F2C
:10695000D4E90A073A1AA8EB0607974228BF174658
:10696000402F1BD905F1400355F8042B9D4240F8F8
:10697000042BF9D1A36A40364033A362D4E90A2339
:106980009A4204D3E16920460439FFF795FF8BF35F
:1069900011884645D9D28AF31188CDE729463A466F
:1069A000FBF792F9A36A3D443E443B44A362E5E70A
:1069B000D0E904239A4217D1C3689BB1836A8BB193
:1069C000043B9B1A0ED01360C368013BC360C369CC
:1069D0001A4483699A42026124BF436A0361002317
:1069E00083620123184670470023FBE700F0CEB80E
:1069F000034B002258631A610222DA60704700BF1D
:106A0000000C0040014B0022DA607047000C00408F
:106A1000014B5863704700BF000C0040014B586A9F
:106A2000704700BF000C00404B6843608B68836078
:106A3000CB68C3600B6943614B6903628B69436236
:106A40000B6803607047000008B5364B40F2FF71D9
:106A50003548D3F888200A43C3F88820D3F8882023
:106A600022F4FF6222F00702C3F88820D3F88820BE
:106A7000D3F8E0200A43C3F8E020D3F808210A4302
:106A8000C3F80821294AD3F808311146FFF7CCFF93
:106A900000F5806002F11C01FFF7C6FF00F5806081
:106AA00002F13801FFF7C0FF00F5806002F15401E8
:106AB000FFF7BAFF00F5806002F17001FFF7B4FF45
:106AC00000F5806002F18C01FFF7AEFF00F58060F9
:106AD00002F1A801FFF7A8FF00F5806002F1C401F0
:106AE000FFF7A2FF00F5806002F1E001FFF79CFFD5
:106AF00000F5806002F1FC01FFF796FF02F58C7152
:106B000000F58060FFF790FF00F0F4F8084B0522D5
:106B1000C3F898204FF06052C3F89C20054AC3F890
:106B2000A02008BD0044025800000258307600083A
:106B300000ED00E01F00080308B500F0D7FAFEF7EB
:106B4000BFFA0F4BD3F8DC2042F04002C3F8DC2040
:106B5000D3F8042122F04002C3F80421D3F8043111
:106B6000084B1A6842F008021A601A6842F00402E0
:106B70001A60FEF7C5FFBDE80840FEF7D5BC00BFB0
:106B8000004402580018024870470000114BD3F827
:106B9000E82042F00802C3F8E820D3F8102142F0C0
:106BA0000802C3F810210C4AD3F81031D36B43F01C
:106BB0000803D363C722094B9A624FF0FF32DA62AF
:106BC00000229A615A63DA605A6001225A611A609F
:106BD000704700BF004402580010005C000C0040E9
:106BE000094A08B51169D3680B40D9B29B076FEA0F
:106BF0000101116107D5202383F31188FEF78CFA78
:106C0000002383F3118808BD000C0040384B4FF07F
:106C1000FF31D3F88020C3F88010D3F88020002201
:106C2000C3F88020D3F88000D3F88400C3F8841020
:106C3000D3F88400C3F88420D3F88400D86F40F0E0
:106C4000FF4040F4FF0040F43F5040F03F00D86761
:106C5000D86F20F0FF4020F4FF0020F43F5020F0D8
:106C60003F00D867D86FD3F888006FEA40506FEACA
:106C70005050C3F88800D3F88800C0F30A00C3F866
:106C80008800D3F88800D3F89000C3F89010D3F8A8
:106C90009000C3F89020D3F89000D3F89400C3F884
:106CA0009410D3F89400C3F89420D3F89400D3F848
:106CB0009800C3F89810D3F89800C3F89820D3F838
:106CC0009800D3F88C00C3F88C10D3F88C00C3F86C
:106CD0008C20D3F88C00D3F89C00C3F89C10D3F818
:106CE0009C10C3F89C20D3F89C3000F0D3B900BFAF
:106CF00000440258614B0122C3F80821604BD3F8CD
:106D0000F42042F00202C3F8F420D3F81C2142F030
:106D10000202C3F81C210222D3F81C31594BDA605D
:106D20005A689104FCD5584A1A6001229A60574A61
:106D3000DA6000221A614FF440429A61514B9A691D
:106D40009204FCD51A6842F480721A604C4B1A6F98
:106D500012F4407F04D04FF480321A6700221A6781
:106D60001A6842F001021A60454B1A685007FCD5B8
:106D700000221A611A6912F03802FBD10121196050
:106D80004FF0804159605A67414ADA62414A1A61BC
:106D90001A6842F480321A60394B1A689103FCD5A4
:106DA0001A6842F480521A601A689204FCD53A4A72
:106DB0003A499A6200225A6319633949DA6399633E
:106DC0005A64384A1A64384ADA621A6842F0A85299
:106DD0001A602B4B1A6802F02852B2F1285FF9D1E1
:106DE00048229A614FF48862DA6140221A622F4A7F
:106DF000DA644FF080521A652D4A5A652D4A9A6519
:106E000032232D4A1360136803F00F03022BFAD1CB
:106E10001B4B1A6942F003021A611A6902F0380228
:106E2000182AFAD1D3F8DC2042F00052C3F8DC2053
:106E3000D3F8042142F00052C3F80421D3F804210E
:106E4000D3F8DC2042F08042C3F8DC20D3F80421E0
:106E500042F08042C3F80421D3F80421D3F8DC20A7
:106E600042F00042C3F8DC20D3F8042142F0004293
:106E7000C3F80421D3F80431704700BF00800051EB
:106E8000004402580048025800C000F0020000010F
:106E90000000FF01008890083220600063020901B1
:106EA0001D02040047040508FD0BFF01200000201F
:106EB0000010E00000010100002000524FF0B0423D
:106EC00008B5D2F8883003F00103C2F8883023B146
:106ED000044A13680BB150689847BDE80840FDF7B5
:106EE000E7B800BF988100204FF0B04208B5D2F853
:106EF000883003F00203C2F8883023B1044A936853
:106F00000BB1D0689847BDE80840FDF7D1B800BF85
:106F1000988100204FF0B04208B5D2F8883003F0D5
:106F20000403C2F8883023B1044A13690BB15069D5
:106F30009847BDE80840FDF7BBB800BF9881002026
:106F40004FF0B04208B5D2F8883003F00803C2F819
:106F5000883023B1044A93690BB1D0699847BDE8E2
:106F60000840FDF7A5B800BF988100204FF0B0425F
:106F700008B5D2F8883003F01003C2F8883023B186
:106F8000044A136A0BB1506A9847BDE80840FDF700
:106F90008FB800BF988100204FF0B04310B5D3F8F0
:106FA000884004F47872C3F88820A30604D5124AF6
:106FB000936A0BB1D06A9847600604D50E4A136BEA
:106FC0000BB1506B9847210604D50B4A936B0BB15C
:106FD000D06B9847E20504D5074A136C0BB1506C8F
:106FE0009847A30504D5044A936C0BB1D06C98471D
:106FF000BDE81040FDF75CB8988100204FF0B04329
:1070000010B5D3F8884004F47C42C3F888206205A8
:1070100004D5164A136D0BB1506D9847230504D55E
:10702000124A936D0BB1D06D9847E00404D50F4A16
:10703000136E0BB1506E9847A10404D50B4A936EA2
:107040000BB1D06E9847620404D5084A136F0BB198
:10705000506F9847230404D5044A936F0BB1D06F47
:107060009847BDE81040FDF723B800BF9881002085
:1070700008B50348FDF7D2F8BDE80840FDF718B899
:10708000D45E002008B5FFF7ABFDBDE80840FDF772
:107090000FB80000062108B50846FDF743F90621A0
:1070A0000720FDF73FF906210820FDF73BF90621EF
:1070B0000920FDF737F906210A20FDF733F90621EB
:1070C0001720FDF72FF906212820FDF72BF90921BC
:1070D0007A20FDF727F907213220FDF723F90C214B
:1070E0005220BDE80840FDF71DB9000008B5FFF7C4
:1070F0008DFD00F00DF8FDF7B9FAFDF791FCFDF7F5
:1071000063FBFFF741FDBDE80840FFF76FBC0000DF
:107110000023054A19460133102BC2E9001102F180
:107120000802F8D1704700BF988100200B46014645
:10713000184600F003B8000000F00EB810B5054C7A
:1071400013462CB10A4601460220AFF3008010BD61
:107150002046FCE700000000024B0146186800F0E2
:1071600035B800BF6422002010B5013902449042B6
:1071700001D1002005E0037811F8014FA34201D0AE
:10718000181B10BD0130F2E72DE9F041A3B1C91A77
:1071900017780144044603F1FF3C8C42204601D994
:1071A000002009E00578BD4204F10104F5D10CEBA3
:1071B0000405D618A54201D1BDE8F08115F8018D6E
:1071C00016F801EDF045F5D0E7E7000037B50029E6
:1071D00044D051F8043C0190002BA1F10404B8BF45
:1071E000E41800F047F81E4A0198136833B9636049
:1071F000146003B0BDE8304000F042B8A34208D9A3
:10720000256861198B4201BF19685B6849192160C3
:10721000EDE71A465B680BB1A342FAD9116855181D
:10722000A5420BD1246821445418A3421160E0D137
:107230001C685B68536021441160DAE702D90C23B3
:107240000360D6E7256861198B4204BF19685B6843
:10725000636004BF491921605460CAE703B030BDC0
:1072600018820020034611F8012B03F8012B002A95
:10727000F9D17047014800F009B800BF1C82002016
:10728000014800F005B800BF1C82002070470000D4
:10729000704700006F72672E6172647570696C6F61
:1072A000742E437562654F72616E67652D706572ED
:1072B000697068004E6F20617070207369670A0002
:1072C000426164206677206C656E6774682025755E
:1072D0000A0042616420626F6172645F6964202504
:1072E000752073686F756C642062652025750A00CF
:1072F0004261642066772064657363726970746F9D
:1073000072206C656E6774682025750A004261649E
:107310002061707020435243203078253038783A0D
:10732000307825303878203078253038783A307801
:10733000253038780A00476F6F64206669726D7770
:107340006172650A0040A2E4F164689106000000E1
:1073500053544D333248373F3F3F0053544D33323F
:10736000483734332F37353300000000F8640020ED
:10737000D45E002043414E464449666163653A202D
:107380004D6573736167652052414D204F7665727C
:10739000666C6F77210000004261642043414E49D2
:1073A0006661636520696E6465782E0000010000E7
:1073B0000001FF0000A0004000A400400000000009
:1073C00000000000C1250008991E0008012D0008DA
:1073D0008D1E0008091F00081923000881200008DD
:1073E000D11E0008D51E0008911E0008AD1E000821
:1073F000951E0008D9220008B91E00080D2E0008AD
:10740000C51E0008AD220008009600000000000024
:10741000000000000000000000000000000000006C
:107420000000000035460008214600085D460008BF
:107430004946000855460008414600082D46000808
:10744000194600086946000800000000454700088A
:10745000314700086D470008594700086547000894
:10746000514700083D4700082947000879470008B0
:107470000000000001000000000000006D61696E66
:107480000000000069646C6500000000847400085E
:1074900080630020F864002001000000BD50000857
:1074A000000000004172647550696C6F74002542E1
:1074B0004F415244252D424C002553455249414CE1
:1074C00025000000020000000000000065490008DF
:1074D000D549000840004000A07D0020B07D00207C
:1074E0000200000000000000030000000000000097
:1074F0001D4A00080000000010000000C07D0020B0
:107500000000000001000000000000004880002092
:1075100001010200C5540008D55300087154000849
:1075200055540008430000002C7500080902430070
:10753000020100C03209040000010202010005241A
:1075400000100105240100010424020205240600A4
:1075500001070582030800FF09040100020A000078
:1075600000070501024000000705810240000000FD
:10757000120000007875000812011001020000409E
:10758000091241570002010203010000040309042B
:1075900025424F415244250030313233343536379D
:1075A00038394142434445460000000000000020B5
:1075B0000000020002000000000100300000000096
:1075C000000000000000002400000800040000008B
:1075D0000004000000FC0000020000000000043075
:1075E00000800000000000000000003800000100E2
:1075F0000100000000000000714B0008294E000847
:10760000D54E00084000400080810020808100208D
:107610000100000090810020800000004001000077
:107620000800000000010000000400000800000045
:107630000000802A00000000AAAAAAAA00000024D4
:10764000FFFF00000000000000A00A00002100026F
:1076500000000000AAAAAAAA00000000FFFF000084
:1076600000000009000009001400005400000000A0
:10767000AAAAAAAA14000054FFFF000000000000FC
:10768000000000000A40100000000000AAAA8AAA18
:1076900000401000FFFF0000990000000000000003
:1076A0000081020000000000AAAAAAAA004101006D
:1076B000FFFF000000000070070000000000000055
:1076C00000000000AAAAAAAA00000000FFFF000014
:1076D00000000000000000000000000000000000AA
:1076E000AAAAAAAA00000000FFFF000000000000F4
:1076F000000000000000000000000000AAAAAAAAE2
:1077000000000000FFFF000000000000000000007B
:107710000000000000000000AAAAAAAA00000000C1
:10772000FFFF00000000000000000000000000005B
:1077300000000000AAAAAAAA00000000FFFF0000A3
:107740000000000000000000000000000000000039
:10775000AAAAAAAA00000000FFFF00000000000083
:10776000000000007C8BFF7F010000000000000093
:10777000780500000000000000001E00000000006E
:10778000FE2A0100D2040000FF00000000000000FB
:10779000507300083F000000500400005B730008B5
:1077A0003F00000000960000000008009600000066
:1077B00000080000040000008C75000800000000B4
:1077C00000000000000000000000000000000000B9
:1077D00000000000682200200000000000000000FF
:1077E0000000000000000000000000000000000099
:1077F0000000000000000000000000000000000089
:107800000000000000000000000000000000000078
:107810000000000000000000000000000000000068
:107820000000000000000000000000000000000058
:08783000000000000000000050
:00000001FF
